:100000000C94D0020C9400000C9400000C9400009E
:100010000C9400000C9400000C9400000C94000060
:100020000C9400000C9400000C9400000C94000050
:100030000C9400000C9400000C9400000C94000040
:100040000C94BF1D0C9400000C9400000C94000054
:100050000C9400000C9400000C9400000C94000020
:100060000C9400000C9400000C9400000C94000010
:100070000C9400000C9400000C946B1E0C94000077
:100080000C94751E0C9400000C94000001000203F7
:1000900053030102040810204080FEFDFBF7EFDF50
:1000A000BF7F252E306600252E316600252E326654
:1000B00000252E336600252E346600252E35660079
:1000C000252E3666000025306C640025316C6400F6
:1000D00025326C640025336C640025346C64002583
:1000E000356C640025366C640025376C6400253857
:1000F0006C640025396C640025306C750025316C0A
:10010000750025326C750025336C750025346C75CF
:100110000025356C750025366C750025376C75002B
:1001200025386C750025396C75004D075C075F0735
:10013000A807BA07C107D207D907E807F7070608D3
:1001400009080C0855085A085F08640869086E0811
:10015000730888088908D00814095B099909B3094C
:10016000C409F809340A480A5C0A740A8C0AA40A09
:10017000B90AC40ACF0ADA0AE50AF00AFD0A070B2F
:10018000110B210B310B410B510B5A0B630B6E0BF7
:10019000790B840B8F0BB20BD50BF80B1B0C3E0CA1
:1001A000610C7A0CB60CE60C2A0D4F0D8E0DC40DA9
:1001B000000E1C0E360E670E970EC60EE50E120FC1
:1001C000430F5A0FAE0FD30FF80F13103C105310FC
:1001D0006A1081109810AF10C610DD10F4100B11CA
:1001E0003C119C11C111E211101228128A12C61280
:1001F00002131F137613B1132E146114D314EE14CB
:100200006F16E7166D1770177C178B17E5175618C2
:10021000C1182F1960198B19D619311A571A871A54
:100220006D176D176D176D176D176D176D176D17AE
:100230006D176D176D176D176D176D176D176D179E
:100240006D176D176D176D176D176D176D176D178E
:100250006D176D176D176D176D176D176D176D177E
:100260006D176D176D176D176D176D176D176D176E
:100270006D176D176D176D176D176D176D176D175E
:100280006D176D176D176D176D176D176D176D174E
:100290006D176D176D176D176D176D176D176D173E
:1002A0006D176D176D176D176D176D176D176D172E
:1002B0006D176D176D176D176D176D176D176D171E
:1002C0006D176D176D176D176D176D176D176D170E
:1002D0006D176D176D176D176D176D176D176D17FE
:1002E0006D176D176D176D176D176D176D176D17EE
:1002F0006D176D176D176D176D176D176D176D17DE
:100300006D176D176D176D176D176D176D176D17CD
:100310006D176D176D176D176D176D176D176D17BD
:100320006D176D176D176D176D176D176D176D17AD
:100330006D176D176D176D176D176D176D176D179D
:100340006D176D176D176D176D176D176D176D178D
:100350006D17E21A451BEF1B0000000000000000B3
:10036000C0C1C1810140C30103C00280C241C601B6
:1003700006C00780C7410500C5C1C4810440CC0147
:100380000CC00D80CD410F00CFC1CE810E400A00C0
:10039000CAC1CB810B40C90109C00880C841D8013E
:1003A00018C01980D9411B00DBC1DA811A401E0038
:1003B000DEC1DF811F40DD011DC01C80DC41140057
:1003C000D4C1D5811540D70117C01680D641D201BE
:1003D00012C01380D3411100D1C1D0811040F0016F
:1003E00030C03180F1413300F3C1F2813240360038
:1003F000F6C1F7813740F50135C03480F4413C0047
:10040000FCC1FD813D40FF013FC03E80FE41FA013D
:100410003AC03B80FB413900F9C1F88138402800DF
:10042000E8C1E9812940EB012BC02A80EA41EE01B5
:100430002EC02F80EF412D00EDC1EC812C40E40156
:1004400024C02580E5412700E7C1E681264022003F
:10045000E2C1E3812340E10121C02080E041A0010D
:1004600060C06180A1416300A3C1A28162406600B7
:10047000A6C1A7816740A50165C06480A4416C0046
:10048000ACC1AD816D40AF016FC06E80AE41AA01BD
:100490006AC06B80AB416900A9C1A881684078003F
:1004A000B8C1B9817940BB017BC07A80BA41BE0135
:1004B0007EC07F80BF417D00BDC1BC817C40B40156
:1004C00074C07580B5417700B7C1B68176407200BF
:1004D000B2C1B3817340B10171C07080B0415000AE
:1004E00090C191815140930153C052809241960135
:1004F00056C057809741550095C1948154409C0146
:100500005CC05D809D415F009FC19E815E405A003E
:100510009AC19B815B40990159C0588098418801DC
:1005200048C0498089414B008BC18A814A404E00B6
:100530008EC18F814F408D014DC04C808C41440055
:1005400084C185814540870147C04680864182013C
:1005500042C043808341410081C18081404048E1E5
:10056000FA3ECDCC4C3D0AD7A33B6F12033A17B7E6
:100570005138ACC5A73601000000010003008C0013
:10058000040002028E001400530A2A011400670AB4
:100590003E0106027B0A52010400AC0D7605000004
:1005A000F894EE27ECBBF1E0F5BFE5BFE0936C00FB
:1005B000F8E1F1BDE1BD8DE0A2E0BB27ED938A95A6
:1005C000E9F780E090E1A0E0B1E0ED930197E9F771
:1005D000EAE7F5E085919591009761F0A591B591D5
:1005E00005901590BF01F00105900D920197E1F77C
:1005F000FB01F0CFEFEFEDBFE0E1EEBFC0E0D2E0F6
:100600000C94F506E8810E94BA320E942625E2E0A9
:10061000E0939B00E8EDE0939A00E6E0E0939D0014
:10062000E0E0E0939800929A0E94C03221F4EFEC4F
:10063000E093990037C0E130A0E0FA0721F4E7E643
:10064000E09399002FC0E230A0E0FA0721F4E3E341
:10065000E093990027C0E330A0E0FA0721F4E2E23A
:10066000E09399001FC0E430A0E0FA0721F4EFE026
:10067000E093990017C0E530A0E0FA0721F4E7E025
:10068000E09399000FC0E630A0E0FA0721F4E3E020
:10069000E093990007C0E730A0E0FA0719F4E1E021
:1006A000E093990049C0E881EA93ECEAFDE0FA930F
:1006B000EA930E942625E2E0EBB9E8EDEAB9E6E02C
:1006C000E0939500E0E0E0939000189A0E94C03219
:1006D00019F4EFECE9B930C0E130A0E0FA0719F401
:1006E000E7E6E9B929C0E230A0E0FA0719F4E3E34C
:1006F000E9B922C0E330A0E0FA0719F4E2E2E9B96F
:100700001BC0E430A0E0FA0719F4EFE0E9B914C027
:10071000E530A0E0FA0719F4E7E0E9B90DC0E630EA
:10072000A0E0FA0719F4E3E0E9B906C0E730A0E079
:10073000FA0711F4E1E0E9B921960895E0E0EBBB96
:10074000EFEFEABBE0E0E5BBEFEFE4BBE0EFE2BBDD
:10075000E3E0E1BBEFE0E0936200E8E0E0936100FA
:10076000E1E0E0936500E0E1E0936400E0E0E0BFF9
:10077000E4E0E3BFE6E0E2BFE0E0E1BFE1E0E7BFE5
:10078000E0E0E0937D00E0E8E8B9E0E0E0BDECE91E
:10079000E0939E0DE091920DEE7FE160E093920D6B
:1007A000E5E6E0939C0DE4E0E0939D0DE0E0E0934E
:1007B000A70DE2E0EA930E9402034424E1E05E2EEA
:1007C000E2E0E0930102E0B3E095AE2FEA2FE2957C
:1007D000EF70E0930002EFE1E1BDEFE0E1BD78945E
:1007E00008950E949A3FE0E0E093510AE093520A94
:1007F000E8E0F0E80E94C4320E94753D2E2F3F2FA2
:100800000E94CD3200E010E00217130710F00C94A4
:10081000E104A6E2BAE0BF93AF930E94663DDF0118
:100820000E94D5323196EA0FFB1FAF91BF91ED9335
:10083000FC93E091260AF091270A0E94793DE1504D
:10084000F040604070404E2F5F2F0E94DC320E94CB
:10085000D532E230A0E0FA0751F50E94E432E0918F
:10086000260AF091270AE491E17079F00E94EC32B7
:10087000FF93EF93E081EF93A2E9B0E00E94F3329F
:10088000AF91EA2BAF91BF910EC00E94EC32FF9363
:10089000EF93E081EF93AAE9B0E00E94F332AF91C9
:1008A000EA23AF91BF91EC930E94DC3275C0E33034
:1008B000A0E0FA0721F0E430A0E0FA0779F40E9402
:1008C000E432A42FB52FAA5FBD4FE091260AF09124
:1008D000270AE491EC930E94DC325EC0E530A0E090
:1008E000FA0721F0E630A0E0FA0789F40E94E4322A
:1008F000E42FF52F0E94FB32E091260AF091270A9F
:100900000E94753DED93FC930E94DC3245C0E730B8
:10091000A0E0FA0721F0E830A0E0FA0709F404C0EB
:10092000E930A0E0FA0789F40E94E432E42FF52FC1
:100930000E940233E091260AF091270A0E94793D35
:100940000E94703D0E94DC3227C0EA30A0E0FA0726
:1009500019F50E94E432E091260AF091270AE49109
:10096000E03081F0E42FF52F4F5F5F4FEA5FFD4FDE
:10097000FF93EF930E94E4323197E491AF91BF91DE
:10098000EC93E9CFA6E0B2E0A40FB51FE0E0EC9352
:100990000E94E4323197E491E091260AF091270A0F
:1009A000E491E13049F4E091510AF091520A319614
:1009B000E093510AF093520A0E94E4320F5F1F4FF6
:1009C00023CF0E94A13F269608951A930A93E52DFE
:1009D000F0E0E130A0E0FA0769F5909800E001301E
:1009E00040F50E940933A9E9BDE00E9410330E943E
:1009F0000933AFE9BDE00E941733A7E9BDE00E94CB
:100A00001733A9EABDE00E941733A8EABDE00E94AF
:100A10001733A7EABDE00E941C33E02F0E94213368
:100A2000FF93EF93E2E0EA93EF91FF9109950F5F57
:100A3000D6CFA7C0E230A0E0FA0711F00C94C105B0
:100A4000E0E0F0E8E093260AF093270A0E942B33B7
:100A50003297FA93EA93E2E0F0E8FA93EA930E947D
:100A6000A325DF01E091260AF091270A0E94753D37
:100A7000EA17FB0711F00C94BE050E94F103EAE0AF
:100A8000F0E80E94C43234900E94E43200E0031582
:100A900010F00C94B505E091260AF091270AE49134
:100AA000EF701E2FE12F0E942133FF93EF93E0910F
:100AB000260AF091270A3196E491EA93EF91FF918B
:100AC00009950E943333A7EABDE0AE0FBF1FE09146
:100AD000260AF091270AE491E295EF70EC930E94C8
:100AE0003333A1EABDE0AE0FBF1F0E942B33ED935D
:100AF000FC930E943333A0EABDE0AE0FBF1FE0912C
:100B0000260AF091270A34960E943A33A3EABDE000
:100B1000AE0FBF1FE091260AF091270A35960E947A
:100B20003A33AAEABDE0AE0FBF1FE091260AF0916A
:100B3000270A3696ED93FC93E091260AF091270A56
:100B40003696FF93EF930E943333A3EABDE00E94F1
:100B50003D330E94613CAF91BF91EA0FFB1FE093D0
:100B6000260AF093270A0F5F92CFE0E0F0E8E093C7
:100B7000260AF093270A909A919803C0E1E05E2E2E
:100B8000919A452C8FC20E949C3F00E010E0E32D1B
:100B9000F0E00E171F0710F00C94F1060E9442338C
:100BA000A8EABDE00E943D33309711F00C94B806DE
:100BB0000E944233AFE9BDE0AE0FBF1FEC91EF934F
:100BC0000E944233A3EABDE0AE0FBF1FEC91AF918C
:100BD000AE1710F00C94AF060E944233AFE9BDE0AF
:100BE0000E943D330E94613C2E2F3F2F0E944233D2
:100BF000AAEABDE00E94493331960E9451333097F2
:100C000011F00C9453060E944233A7EABDE00E9403
:100C10003D333097F9F40E944233AAEABDE00E94C6
:100C200056330E945F33AAEABDE00E9449330E9416
:100C300062330E945F33AAEABDE00E9449330E94FA
:100C40006E33AAEABDE00E9449330E947A330E94C3
:100C5000803322C0E130A0E0FA07F1F40E94423371
:100C6000AAEABDE00E9456330E944233AAEABDE0E0
:100C70000E9449330E9462330E944233AAEABDE0D7
:100C80000E9449330E946E33AAEABDE00E944933B4
:100C90000E947A330E9486330E944233A9EABDE063
:100CA0000E948C3355C0E130A0E0FA0711F00C949B
:100CB000A8060E944233A7EABDE00E943D33309768
:100CC000F9F40E944233AAEABDE00E9456330E9422
:100CD0005F33AAEABDE00E9449330E9462330E945A
:100CE0005F33AAEABDE00E9449330E946E33AAEA4C
:100CF000BDE00E9449330E947A330E94913322C0A2
:100D0000E130A0E0FA07F1F40E944233AAEABDE024
:100D10000E9456330E944233AAEABDE00E94493342
:100D20000E9462330E944233AAEABDE00E94493326
:100D30000E946E33AAEABDE00E9449330E947A33D2
:100D40000E9497330E944233A9EABDE00E949D337E
:100D50000E944233AFE9BDE00E94A23307C00E9467
:100D60004233AFE9BDE0AE0FBF1FE0E0EC9336C009
:100D7000E530A0E0FA0729F40E9442330E94A7332D
:100D80002DC0E630A0E0FA0749F50E944233A7E9FA
:100D9000BDE00E94A233EC93EF930E944233A0EA9D
:100DA000BDE0AE0FBF1FEC91AF91AE1748F40E94AB
:100DB0004233AFE9BDE0AE0FBF1FEC91E15007C079
:100DC0000E944233A7E9BDE0AE0FBF1FE0E0EC9305
:100DD0000E944233A8EABDE00E941C330F5F1F4F00
:100DE000D6CE0E94A33F249608950E949E030E949F
:100DF000BD1C0E94211DE52DA42D0E947F3CEF9378
:100E0000A091A80DE0E00E94843CAF91EA2B11F480
:100E10000C944907E42DF0E0E130A0E0FA0711F569
:100E200000E0013080F40E940933A8EABDE0AE0F73
:100E3000BF1FAC91A53029F4E02F0E94AD330E9472
:100E4000A7330F5FEECFE0916300E17039F4A0911A
:100E50000102A23011F4E2E05E2E03C0E2E0E09372
:100E6000010216C0E230A0E0FA0791F40E94121CC1
:100E70000E94C305E0916300E170EF93A09101022D
:100E8000E1E00E947F3CAF91EA2B11F0E1E05E2EA1
:100E900002C00E94E504ADCFFFCFE1E0F0E060E0EA
:100EA00070E0E093490AF0934A0A60934B0A70930A
:100EB0004C0A0E94DC3208950E94DC3208950E94A0
:100EC000B3330E94B63317FF21C010700E94BC33A9
:100ED000E081EF930E94C533AF91EA2369F0E1E02E
:100EE000F0E060E070E0E093490AF0934A0A609312
:100EF0004B0A70934C0A09C0E0E0E093490AE09382
:100F00004A0AE0934B0AE0934C0A21C0015010407A
:100F10000E94CF33E081EF930E94C533AF91EA2363
:100F200069F0E1E0F0E060E070E0E093490AF093FE
:100F30004A0A60934B0A70934C0A09C0E0E0E093C0
:100F4000490AE0934A0AE0934B0AE0934C0AAAC08C
:100F50000E94DC320E94D633F0E0E7FDFFEF0E94F2
:100F6000753CE093490AF0934A0A60934B0A7093E8
:100F70004C0A08950E94DC320E94D6330E94DE3370
:100F800008950E94DC320E94EA330E94663D0E946E
:100F9000753CE093490AF0934A0A60934B0A7093B8
:100FA0004C0A08950E94DC320E94EA330E94EF331B
:100FB00008950E94DC320E94FC330E946A3DE09357
:100FC000490AF0934A0A60934B0A70934C0A0895B9
:100FD0000E94DC320E94FC330E946A3DE093490A81
:100FE000F0934A0A60934B0A70934C0A08950E944A
:100FF000DC320E94FC330E946A3DE0934D0AF0937C
:101000004E0A60934F0A7093500A08950E94DC3292
:1010100008950E94DC3208950E94B3330E94B633D3
:1010200017FF20C01070E091490AE17069F00E943A
:10103000BC33FF93EF93E081EF930E94C533AF91F0
:10104000EA2BAF91BF910CC00E94BC33FF93EF938A
:10105000E081EF930E940134AF91EA23AF91BF91F9
:10106000EC9320C001501040E091490AE17069F012
:101070000E94CF33FF93EF93E081EF930E94C5333B
:10108000AF91EA2BAF91BF910CC00E94CF33FF9379
:10109000EF93E081EF930E940134AF91EA23AF9187
:1010A000BF91EC930991199108950E94DC320E943E
:1010B0000B3408950E94DC320E940B3408950E9484
:1010C000DC320E941C3408950E94DC320E941C34E1
:1010D00008950E94DC320E94313408950E94DC326F
:1010E0000E94313408950E94DC320E944634A6E00A
:1010F000B2E00E94633CAE0FBF1FE0914D0AF09139
:101100004E0A60914F0A7091500A0E94703D0895F6
:10111000089524970E94B3330E94E4320E944B3416
:1011200041F1EFEFFFEF6FEF7FEFEA83FB836C831B
:101130007D8300E0011760F40E946A340E947234DB
:101140000E94243CEA83FB836C837D830F5FF2CF94
:101150000E9488340E949534E1E0F0E060E070E0A5
:10116000E093490AF0934A0A60934B0A70934C0A41
:1011700012C0A6E2BAE0BF93AF930E949F34AF9132
:10118000BF910E94A93429F00E946A340E949534CC
:1011900002C00E94DC320E946A340E94953487C0EB
:1011A00024970E94B3330E94E4320E944B3429F109
:1011B000E0E0EA83EB83EC83ED8300E0011760F469
:1011C0000E946A340E9472340E94293CEA83FB83A5
:1011D0006C837D830F5FF2CF0E9488340E94953428
:1011E000E1E0F0E060E070E0E093490AF0934A0A41
:1011F00060934B0A70934C0A12C0A6E2BAE0BF9308
:10120000AF930E949F34AF91BF910E94A93429F0FF
:101210000E946A340E94953402C00E94DC320E940F
:101220006A340E94953443C024970E94B3330E94CD
:10123000E4320E944B3429F1E0E0EA83EB83EC8353
:10124000ED8300E0011760F40E946A340E9472345A
:101250000E942E3CEA83FB836C837D830F5FF2CF79
:101260000E9488340E949534E1E0F0E060E070E094
:10127000E093490AF0934A0A60934B0A70934C0A30
:1012800012C0A6E2BAE0BF93AF930E949F34AF9121
:10129000BF910E94A93429F00E946A340E949534BB
:1012A00002C00E94DC320E946A340E949534198187
:1012B0000881269608950E94DC320E946A340E94BA
:1012C000B3340E94823FF9F00E946A340E94B33422
:1012D0000E947A3CE093490AF0934A0A60934B0AD1
:1012E00070934C0A0E946A340E949534E1E0F0E069
:1012F00060E070E0E093490AF0934A0A60934B0A79
:1013000070934C0A11C00E94DC32E091260AF091E1
:10131000270A0E94753DF07829F00E946A340E94E5
:10132000953402C00E94DC320E946A340E949534D7
:1013300008950E94DC320E946A340E94B3340E94F5
:10134000823F71F0E0E0E093490AE0934A0AE093BB
:101350004B0AE0934C0A0E946A340E94953402C002
:101360000E94DC3208950E94DC320E946A340E949E
:10137000B3340E94823F29F00E946A340E9495345F
:1013800002C00E94DC3208950E94DC320E946A345E
:101390000E94B3340E94823F11F10E946A340E947D
:1013A000B3340E94823F89F4E1E0F0E060E070E055
:1013B000E093490AF0934A0A60934B0A70934C0AEF
:1013C0000E94C5340E94953409C0E0E0E093490AC8
:1013D000E0934A0AE0934B0AE0934C0A04C00E944F
:1013E0006A340E9495340E946A340E9495340895AC
:1013F0000E94DC320E946A340E94B3340E94823F11
:1014000009F50E946A340E94B3340E94823FC9F0F9
:10141000E0E0E093490AE0934A0AE0934B0AE09344
:101420004C0A0E94C5340E949534E1E0F0E060E08F
:1014300070E0E093490AF0934A0A60934B0A709374
:101440004C0A0DC00E946A340E949534E0E0E0939B
:10145000490AE0934A0AE0934B0AE0934C0A0E943F
:101460006A340E949534089524970E94DC320E94C9
:101470006A340E94B334E883F9836A837B830E94D1
:101480006A340E94B3340E94CD340E9495346FC0F8
:1014900024970E94DC320E946A340E94B334E883AD
:1014A000F9836A837B830E946A340E94B3340E946A
:1014B000DF340E9495345BC024970E94DC320E9486
:1014C0006A340E94B334E883F9836A837B830E9481
:1014D0006A340E94B334A881B9818A819B810E94B9
:1014E000F1340E94953443C024970E94DC320E945C
:1014F0006A340E94B334E883F9836A837B830E9451
:101500006A340E94B334A881B9818A819B810E9488
:10151000FF340E9495342BC024970E94DC320E9435
:101520006A340E94B334E883F9836A837B830E9420
:101530006A340E94B334A881B9818A819B810E9458
:101540000D350E94953413C024970E94DC320E940E
:101550006A340E94B334E883F9836A837B830E94F0
:101560006A340E94B3340E941B350E94953424963D
:1015700008950E94DC320E946A340E942D350E9438
:1015800043350E94953408950E94DC320E946A34EB
:101590000E942D350E9451350E94953408950E9475
:1015A000DC320E946A340E942D350E94F1340E9480
:1015B000953408950E94DC320E946A340E942D35D1
:1015C0000E94FF340E94953408950E94DC320E94EC
:1015D0006A340E942D350E940D350E94953408957D
:1015E0000E94DC320E946A340E942D350E94A13C88
:1015F0000E945F350E949534089524970E94DC3242
:101600000E946B350E94CD340E94953446C22497C7
:101610000E94DC320E946B350E94DF340E949534B8
:101620003CC224970E94DC320E946B35A881B981AC
:101630008A819B810E94763F0E945F350E9495348B
:101640002CC224970E94DC320E946B35A881B9819C
:101650008A819B810E947C3F0E945F350E94953465
:101660001CC224970E94DC320E946B35A881B9818C
:101670008A819B810E946A3F0E945F350E94953457
:101680000CC224970E94DC320E946B35A881B9817C
:101690008A819B810E94703F0E945F350E94953431
:1016A000FCC10E94DC320E9484350E9443350E94B6
:1016B000953408950E94DC320E9484350E94513591
:1016C0000E94953408950E94DC320E9484350E9465
:1016D000763F0E945F350E94953408950E94DC3267
:1016E0000E9484350E947C3F0E945F350E949534A1
:1016F00008950E94DC320E9484350E946A3F0E9455
:101700005F350E94953408950E94DC320E94843532
:101710000E94703F0E945F350E94953408950E9498
:10172000DC320E946A340E94B3340E94823F99F0F6
:101730000E946A340E9493350E945508E1E0F0E06F
:1017400060E070E0E093490AF0934A0A60934B0A24
:1017500070934C0A02C00E949D350E946A340E9418
:10176000953408950E94DC320E946A340E94B3349A
:101770000E94823F99F00E946A340E9493350E9431
:101780005F08E1E0F0E060E070E0E093490AF09388
:101790004A0A60934B0A70934C0A02C00E949D351E
:1017A0000E946A340E94953408950E94DC320E949F
:1017B0006A340E94B3340E94823F99F00E946A34D6
:1017C0000E9493350E946908E1E0F0E060E070E07B
:1017D000E093490AF0934A0A60934B0A70934C0ACB
:1017E00002C00E949D350E946A340E94953408957B
:1017F0000E94DC320E946A340E94B3340E94823F0D
:1018000099F00E946A340E9493350E945A08E1E0E0
:10181000F0E060E070E0E093490AF0934A0A6093D8
:101820004B0A70934C0A02C00E949D350E946A3494
:101830000E94953408950E94DC320E946A340E940E
:10184000B3340E94823F99F00E946A340E9493351B
:101850000E946408E1E0F0E060E070E0E093490A93
:10186000F0934A0A60934B0A70934C0A02C00E949C
:101870009D350E946A340E94953408950E94DC329E
:101880000E946A340E94B3340E94823F99F00E9401
:101890006A340E9493350E946E08E1E0F0E060E057
:1018A00070E0E093490AF0934A0A60934B0A709300
:1018B0004C0A02C00E949D350E946A340E949534F1
:1018C00008950E94DC320E946A340E94B3340E9460
:1018D000823F49F00E946A340E94B3340E944B3E1A
:1018E0000E94A53502C00E949D350E946A340E9464
:1018F0009534089524970E94B3330E94E4320E94E5
:101900004B3429F1E0E0EA83EB83EC83ED8300E0E4
:10191000011760F40E946A340E9472340E941A3CDB
:10192000EA83FB836C837D830F5FF2CF0E94883450
:101930000E949534E1E0F0E060E070E0E093490A55
:10194000F0934A0A60934B0A70934C0A0AC0A6E2CD
:10195000BAE0BF93AF930E94BC35AF91BF91ED93B6
:10196000FC930E946A340E9495340AC124970E9415
:10197000B3330E94E4320E944B34C9F0E0E0EA83C2
:10198000EB83EC83ED8300E0011750F40E94C73530
:101990000E94893EEA83FB836C837D830F5FF4CFD3
:1019A000EA81FB816C817D810E94A5350AC0A6E297
:1019B000BAE0BF93AF930E94BC35AF91BF91ED9356
:1019C000FC930E946A340E949534DAC024970E94E6
:1019D000DC320E946A340E94B3340E94823F99F143
:1019E0000E946A340E94B334E883F9836A837B835C
:1019F0000E946A340E949335A091490AB0914A0A24
:101A000080914B0A90914C0AE881F9816A817B812F
:101A10000E941F3CE093490AF0934A0A60934B0AE4
:101A200070934C0A0E946A340E949534E1E0F0E021
:101A300060E070E0E093490AF0934A0A60934B0A31
:101A400070934C0A02C00E94D6350E946A340E94EC
:101A5000953423C024970E94DC320E946A340E948D
:101A6000B3340E94823F99F00E94DE35A0914D0A66
:101A7000B0914E0A80914F0A9091500AE881F98105
:101A80006A817B810E94823E0E94A53502C00E942D
:101A9000D6350E946A340E9495342496089524977E
:101AA0000E94B3330E94E4320E944B3441F1E1E0E2
:101AB000F0E060E070E0EA83FB836C837D8300E00C
:101AC000011760F40E946A340E9472340E94E63C5E
:101AD000EA83FB836C837D830F5FF2CF0E9488349F
:101AE0000E949534E1E0F0E060E070E0E093490AA4
:101AF000F0934A0A60934B0A70934C0A0AC0A6E21C
:101B0000BAE0BF93AF930E94BC35AF91BF91ED9304
:101B1000FC930E946A340E94953432C024970E943C
:101B2000B3330E94E4320E944B34E1F0E0E0F0E095
:101B300060E87FE3EA83FB836C837D8300E0011729
:101B400050F40E94C7350E94D73EEA83FB836C8322
:101B50007D830F5FF4CFEA81FB816C817D810E94E0
:101B6000A5350AC0A6E2BAE0BF93AF930E94BC3588
:101B7000AF91BF91ED93FC930E946A340E9495341B
:101B8000198108812696089524970E94DC320E94CC
:101B90006A340E94B3340E94823F59F10E946A3431
:101BA0000E94B334E883F9836A837B830E946A349A
:101BB0000E94B334A881B9818A819B810E94243D0F
:101BC000E093490AF0934A0A60934B0A70934C0AD7
:101BD0000E946A340E949534E1E0F0E060E070E039
:101BE000E093490AF0934A0A60934B0A70934C0AB7
:101BF00002C00E94D6350E946A340E94953411C2F8
:101C000024970E94DC320E946A340E94B3340E94FE
:101C1000823F59F00E946B35A881B9818A819B81EE
:101C20000E94093F0E94A53502C00E94D6350E943D
:101C30006A340E949534F5C124970E94DC320E94D8
:101C40006A340E94B3340E94823F49F00E94DE351C
:101C50000E94EE350E94942D0E94A53502C00E947C
:101C6000D6350E946A340E949534DBC10E94DC3272
:101C70000E946A340E94B3340E94823F09F10E949C
:101C80006A340E94B334EF5FFF4F6F4F7F4FE09392
:101C9000490AF0934A0A60934B0A70934C0A0E94D7
:101CA0006A340E949534E1E0F0E060E070E0E09397
:101CB000490AF0934A0A60934B0A70934C0A02C097
:101CC0000E949D350E946A340E94953408950E94B6
:101CD000DC320E946A340E94B3340E94823F01F1D8
:101CE0000E946A340E94B334319760407040E093A0
:101CF000490AF0934A0A60934B0A70934C0A0E9477
:101D00006A340E949534E1E0F0E060E070E0E09336
:101D1000490AF0934A0A60934B0A70934C0A02C036
:101D20000E949D350E946A340E94953408950E9455
:101D3000DC320E946A340E94B3340E94823FF9F080
:101D40000E946A340E94B3340E94373CE093490AEF
:101D5000F0934A0A60934B0A70934C0A0E946A34CB
:101D60000E949534E1E0F0E060E070E0E093490A21
:101D7000F0934A0A60934B0A70934C0A02C00E9487
:101D80009D350E946A340E94953408950E94DC3289
:101D90000E946A340E94B3340E94823F79F00E940C
:101DA000F707E0914D0AF0914E0A60914F0A709149
:101DB000500A0E94EF3D0E94A53502C00E949D3549
:101DC0000E946A340E94953408950E94DC320E9479
:101DD0006A340E94B3340E94823FE9F00E949C3230
:101DE0000E94753CE093490AF0934A0A60934B0ABB
:101DF00070934C0A0E946A340E949534E1E0F0E04E
:101E000060E070E0E093490AF0934A0A60934B0A5D
:101E100070934C0A02C00E94DC320E946A340E9415
:101E2000953408950E94DC320E946A340E94B334D3
:101E30000E94823F09F10E946A340E94B3340E94DA
:101E40007F3D0E94692DE093490AF0934A0A60930E
:101E50004B0A70934C0A0E946A340E949534E1E068
:101E6000F0E060E070E0E093490AF0934A0A609382
:101E70004B0A70934C0A02C00E949D350E946A343E
:101E80000E94953408950E94DC320E946A340E94B8
:101E9000B3340E94823F39F00E94FF350E948E2D9C
:101EA0000E94A53502C00E949D350E946A340E949E
:101EB0009534089524970E94DC320E946A340E946F
:101EC000B3340E94823F11F40C94A70F0E94FF3597
:101ED0000E94073CE883F9836A837B83A0914D0AC3
:101EE000B0914E0A80914F0A9091500A0E940C3690
:101EF0000E944A3F28F4E881F9816A817B810CC005
:101F0000E0914D0AF0914E0A60914F0A7091500A8B
:101F10000E947F3D0E940D3C0E94183EE093490ABA
:101F2000F0934A0A60934B0A70934C0A0E946A34F9
:101F30000E949534E1E0F0E060E070E0E093490A4F
:101F4000F0934A0A60934B0A70934C0A02C00E94B5
:101F50009D350E946A340E94953463C00E94DC3231
:101F60000E946A340E94B3340E94823FA9F00E940A
:101F7000FF350E940D3C0E9417360E949534E1E027
:101F8000F0E060E070E0E093490AF0934A0A609361
:101F90004B0A70934C0A02C00E949D350E946A341D
:101FA0000E94953408950E94DC320E946A340E9497
:101FB000B3340E94823FA9F00E94FF350E94073C83
:101FC0000E9417360E949534E1E0F0E060E070E096
:101FD000E093490AF0934A0A60934B0A70934C0AC3
:101FE00002C00E949D350E946A340E949534089573
:101FF00024970E94DC320E946A340E94B3340E940B
:10200000823F49F00E94DE350E94EE350E942A2F61
:102010000E94A53502C00E94D6350E946A340E94F3
:102020009534249608950E94DC320E946A340E94FE
:10203000B3340E94823FC9F00E946A340E94B334D4
:102040000E947F3D0E947A2D0E9422360E94953484
:10205000E1E0F0E060E070E0E093490AF0934A0AC2
:1020600060934B0A70934C0A02C00E949D350E94F7
:102070006A340E94953408950E94DC320E946A34CA
:102080000E94B3340E94823F39F00E94FF350E94C3
:10209000A23B0E94A53502C00E949D350E946A3471
:1020A0000E94953408950E94DC320E946A340E9496
:1020B000B3340E94823F39F00E94FF350E947E2E89
:1020C0000E94A53502C00E949D350E946A340E947C
:1020D000953408950E94DC320E946A340E94B33421
:1020E0000E94823F39F00E94FF350E94E22D0E943B
:1020F000A53502C00E949D350E946A340E94953425
:1021000008950E94DC320E946A340E94B3340E9417
:10211000823F39F00E94FF350E948A2F0E94A53528
:1021200002C00E949D350E946A340E949534089531
:102130000E94DC320E946A340E94B3340E94823FC3
:1021400039F00E94FF350E941B300E94A53502C065
:102150000E949D350E946A340E94953408950E9421
:10216000DC320E946A340E94B3340E94823F39F00C
:102170000E94FF350E942A300E94A53502C00E94AD
:102180009D350E946A340E94953408950E94DC3285
:102190000E946A340E94B3340E94823F39F00E9448
:1021A000FF350E94E3300E94A53502C00E949D3594
:1021B0000E946A340E94953408950E94DC320E9485
:1021C0006A340E94B3340E94823F39F00E94FF3586
:1021D0000E9452310E94A53502C00E949D350E9486
:1021E0006A340E94953408950E94DC320E946A3459
:1021F0000E94B3340E94823F39F00E94FF350E9452
:1022000078310E94A53502C00E949D350E946A3433
:102210000E94953408950E94DC320E946A340E9424
:10222000B3340E94823F09F1E091850CF091860C55
:102230006091870C7091880CE093490AF0934A0AE8
:1022400060934B0A70934C0A0E946A340E94953442
:10225000E1E0F0E060E070E0E093490AF0934A0AC0
:1022600060934B0A70934C0A02C00E94DC320E94B9
:102270006A340E949534089524970E94DC320E94AB
:102280006A340E94B3340E94823F11F40C94871187
:102290000E946A340E949335A091490AB0914A0A7B
:1022A00080914B0A90914C0AE091850CF091860C3C
:1022B0006091870C7091880C0E941F3CE883F98321
:1022C0006A837B830E946A340E94B3340E941B3568
:1022D0000E949534E881F9816A817B81E093490A03
:1022E000F0934A0A60934B0A70934C0A0E946A3436
:1022F0000E949534E1E0F0E060E070E0E093490A8C
:10230000F0934A0A60934B0A70934C0A10C00E94E3
:102310002D360E94A93439F00E946A340E94953407
:102320000E94333602C00E942D36ED93FC930E942A
:102330006A340E94953481C10E94DC320E946A3462
:102340000E94B3340E94823FA9F00E946A340E9426
:1023500093350E946A340E949534E1E0F0E060E039
:1023600070E0E093490AF0934A0A60934B0A709335
:102370004C0A02C00E949D350E946A340E94953426
:1023800008950E94DC320E946A340E94B3340E9495
:10239000823F89F00E94F7070E947308E1E0F0E0B5
:1023A00060E070E0E093490AF0934A0A60934B0AB8
:1023B00070934C0A02C00E949D350E946A340E94AC
:1023C000953408950E94DC320E946A340E94B3342E
:1023D0000E94823FF1F00E94DC3234970E94793DE6
:1023E000E093490AF0934A0A60934B0A70934C0AAF
:1023F0000E946A340E949534E1E0F0E060E070E011
:10240000E093490AF0934A0A60934B0A70934C0A8E
:1024100002C00E949D350E946A340E94953408953E
:102420000E94DC320E946A340E94B3340E94823FD0
:1024300041F00E94DC3234970E94793D0E94A5351C
:1024400002C00E949D350E946A340E94953408950E
:1024500022970E949A3F26E032E00E94DC320E94DE
:102460006A340E94B3340E94823F11F40C948012AB
:102470000E946A340E9493350091490A10914A0AD9
:102480000E946A340E949335E091490AF0914A0A09
:10249000EE83FF83E091260AF091270A0E94753DA2
:1024A0000E0F1F1F0E94DC320E946A340E94933577
:1024B000E091490AF0914A0A2E0F3F1F40E050E098
:1024C000EE81FF814E175F0770F4E42FF52F0E9415
:1024D00039363196E050F048E00FF11FE491EC936B
:1024E0004F5F5F4FEDCFE1E0F0E060E070E0E09340
:1024F000490AF0934A0A60934B0A70934C0A02C04F
:102500000E943F360E946A340E9495340E94A13F87
:102510002896089524970E94DC320E946A340E9413
:10252000B3340E94823F59F10E946A340E94B3344E
:10253000E883F9836A837B830E946A340E94B33400
:10254000A881B9818A819B810E94553CE093490A08
:10255000F0934A0A60934B0A70934C0A0E946A34C3
:102560000E949534E1E0F0E060E070E0E093490A19
:10257000F0934A0A60934B0A70934C0A02C00E947F
:10258000D6350E946A340E94953457C024970E9421
:10259000DC320E946A340E94B3340E94823F59F1B7
:1025A0000E946A340E94B334E883F9836A837B8390
:1025B0000E946A340E94B334A881B9818A819B81C8
:1025C0000E94493CE093490AF0934A0A60934B0AFF
:1025D00070934C0A0E946A340E949534E1E0F0E066
:1025E00060E070E0E093490AF0934A0A60934B0A76
:1025F00070934C0A02C00E94D6350E946A340E9431
:1026000095341BC024970E94DC320E946A340E94D9
:10261000B3340E94823F59F00E94DC320E9446345B
:102620000E9447360E9496310E94A53502C00E9442
:102630009D350E946A340E949534249608950A9329
:102640000E94DC320E946A340E94B3340E94823FAE
:1026500011F40C946E130E94F7070E946A340E94D2
:1026600093350091490AE6E0E01708F406E00E947D
:10267000DC320E94463466277727E093490AF093BC
:102680004A0A60934B0A70934C0A0E945236E2EA5F
:10269000F0E0FF93EF930E945F36AF91BF91EA0F96
:1026A000FB1FFA93EA93E0914D0AF0914E0A609174
:1026B0004F0A7091500A0E947F3D84E00E941D2CB9
:1026C0002896E1E0F0E060E070E0E093490AF093E2
:1026D0004A0A60934B0A70934C0A02C00E94D63596
:1026E0000E946A340E949534099108950E94DC3258
:1026F0000E946A340E94B3340E94823F51F1A8E4E0
:10270000BAE0EC91F0E0EF5FEC93E1500E946636A6
:10271000DF01E6E2FAE082E00E94C83D0E946C36EA
:1027200020FE05C00E94CD320E947936F9CF689410
:1027300020F8E091480AE150E093480AEF5FA8E4EE
:10274000BAE0EC910E946636A6E2BAE082E00E940E
:10275000C83DA6E2BAE00E94663D3496ED93FC9334
:10276000089526970E94DC320E946A340E94B33496
:102770000E94823F11F40C9427140E946A34E330C3
:10278000A0E0FA0721F0E430A0E0FA07C9F40E94C3
:102790006A340E94B334E883F9836A837B830E949E
:1027A0006A340E949335E091490AF0914A0AEC8319
:1027B000FD83AC81BD811197E8810E94B93D3AC08B
:1027C000E530A0E0FA0721F0E630A0E0FA07E1F4F6
:1027D0000E946A340E94B334E883F9836A837B835E
:1027E0000E946A340E949335E091490AF0914A0AA6
:1027F000EE0FFF1FEC83FD83AC81BD811297E88152
:10280000F9810E94B13D16C0E730A0E0FA0721F03F
:10281000E830A0E0FA0771F40E946A340E94B334F1
:10282000E883F9836A837B830E946A340E9493352C
:102830000E948636E1E0F0E060E070E0E093490A53
:10284000F0934A0A60934B0A70934C0A02C00E94AC
:102850009D350E946A340E94953431C026970E94AB
:10286000DC320E946A340E94B3340E94823F09F134
:102870000E94F707E0914D0AF0914E0A60914F0ACD
:102880007091500AE883F9836A837B830E946A34DB
:102890000E9493350E948636E1E0F0E060E070E04F
:1028A000E093490AF0934A0A60934B0A70934C0AEA
:1028B00002C00E949D350E946A340E94953426967B
:1028C000089522970E94DC320E946A340E94B33439
:1028D0000E94823F11F40C94CC140E946A340E942E
:1028E00093350E946A34E330A0E0FA0721F0E43027
:1028F000A0E0FA0771F4E091490AF0914A0AE883EE
:10290000F983A881B98111970E949A3D0E94DE3314
:1029100032C0E530A0E0FA0721F0E630A0E0FA0787
:10292000C1F4E091490AF0914A0AEE0FFF1FE883D3
:10293000F983A881B98112970E94963D662777276F
:10294000E093490AF0934A0A60934B0A70934C0A49
:1029500012C0E730A0E0FA0721F0E830A0E0FA0763
:1029600051F40E949836E093490AF0934A0A609322
:102970004B0A70934C0A0E946A340E949534E1E03D
:10298000F0E060E070E0E093490AF0934A0A609357
:102990004B0A70934C0A02C00E949D350E946A3413
:1029A0000E94953419C022970E94DC320E946A343A
:1029B0000E94B3340E94823F49F00E946A340E9410
:1029C00093350E9498360E94A53502C00E949D351D
:1029D0000E946A340E94953422960895EC970E94D2
:1029E000DC320E946A340E94B3340E94823F11F4A8
:1029F0000C9462160E946A340E94B334ECABFDABB7
:102A00006EAB7FAB0E946A340E94B334E8ABF9AB83
:102A10006AAB7BAB0E946A340E94B334ECA7FDA77B
:102A20006EA77FA70E946A340E94B334E8A7F9A773
:102A30006AA77BA70E946A340E94B334ECA3FDA36B
:102A40006EA37FA30E946A340E94B334E8A3F9A363
:102A50006AA37BA30E946A340E94B334EC8FFD8F7B
:102A60006E8F7F8F0E946A340E94B334E88FF98F93
:102A70006A8F7B8F0E946A340E94B334EC8BFD8B8B
:102A80006E8B7F8B0E946A340E94B334EC87FD8783
:102A90006E877F87A091850CB091860C8091870C02
:102AA0009091880C0E94843D0E941F3CE88BF98B1A
:102AB0006A8B7B8BE091850CF091860C6091870C82
:102AC0007091880CEC87FD876E877F87A889B9890C
:102AD0008A899B890E948A3F44F0E1E0F0E060E04F
:102AE00070E0E88BF98B6A8B7B8BA8A9B9A98AA9BE
:102AF0009BA9ECA9FDA96EA97FA90E941F3CE8AF84
:102B0000F9AF6AAF7BAFACA5BDA58EA59FA50E940E
:102B1000E63CE887F9876A877B87E889F9896A89CB
:102B20007B89A8ADB9AD8AAD9BAD0E94E63CA8A556
:102B3000B9A58AA59BA50E94E63CA88DB98D8A8D72
:102B40009B8D0E941A3CEC83FD836E837F83EC8D0A
:102B5000FD8D6E8D7F8DAC81BD818E819F810E94A8
:102B6000903F24F4EC83FD836E837F83E8A1F9A179
:102B70006AA17BA1AC81BD818E819F810E94953F1E
:102B800024F4EC83FD836E837F83AC89BD898E89B9
:102B90009F89E8ADF9AD6AAD7BAD0E941F3CACA149
:102BA000BDA18EA19FA10E94E63CDF01CB01E88977
:102BB000F9896A897B890E94243DE883F9836A83C5
:102BC0007B83EC81FD816E817F81A885B9858A85B3
:102BD0009B850E94A636E093490AF0934A0A6093C7
:102BE0004B0A70934C0AEC8DFD8D6E8D7F8DA091FC
:102BF000490AB0914A0A80914B0A90914C0A0E946E
:102C0000903F44F4E093490AF0934A0A60934B0AD8
:102C100070934C0AE8A1F9A16AA17BA1A091490A8D
:102C2000B0914A0A80914B0A90914C0A0E94953FBC
:102C300044F4E093490AF0934A0A60934B0A709374
:102C40004C0A0E946A340E949534EC81FD816E81A9
:102C50007F81E093490AF0934A0A60934B0A70938C
:102C60004C0A0E946A340E949534E8ADF9AD6AAD11
:102C70007BADE093490AF0934A0A60934B0A709344
:102C80004C0A0E946A340E949534EC85FD856E855D
:102C90007F85E093490AF0934A0A60934B0A709348
:102CA0004C0A0E946A340E949534E1E0F0E060E052
:102CB00070E0E093490AF0934A0A60934B0A7093DC
:102CC0004C0A07C0A6E2BAE00E94663DF896ED9372
:102CD000FC930E946A340E949534EC9608952497E0
:102CE0000A930E94DC320E946A340E94B3340E942C
:102CF000823F11F40C94DE160E94DC320E944634AE
:102D000066277727E983FA836B837C830E946A3482
:102D10000E9493350091490AE9E0E01708F409E0C0
:102D20000E946A34E330A0E0FA0721F0E530A0E029
:102D3000FA0709F404C0E730A0E0FA0789F40E941A
:102D4000AF36E6ECF0E0FF93EF930E945F36AF9171
:102D5000BF910E94B83684E00E945E2D28961DC067
:102D6000E430A0E0FA0721F0E630A0E0FA0709F429
:102D700004C0E830A0E0FA0781F40E94AF36E8EF23
:102D8000F0E0FF93EF930E945F36AF91BF910E94F6
:102D9000B83684E00E945E2D28960E946A340E9414
:102DA0009534E1E0F0E060E070E0E093490AF093F0
:102DB0004A0A60934B0A70934C0A02C00E94D635AF
:102DC0000E946A340E9495340881259608952497BC
:102DD0000E94B3330E946A340E94B3340E94823F3F
:102DE00011F40C946317E091260AF091270A3396A8
:102DF0000491E02FF0E00E94B334EA83FB836C83FC
:102E00007D830E946A340E9493351091490AE9E05B
:102E1000E11708F419E00E94DC320E94463466276C
:102E20007727E093490AF0934A0A60934B0A70931C
:102E30004C0AE02FF0E0E330A0E0FA0721F0E530A3
:102E4000A0E0FA0709F404C0E730A0E0FA0789F42B
:102E50000E945236E6ECF0E0FF93EF930E94C336F7
:102E6000AF91BF910E94CA3684E00E941D2C289623
:102E70001DC0E430A0E0FA0721F0E630A0E0FA0738
:102E800009F404C0E830A0E0FA0781F40E94523649
:102E9000E8EFF0E0FF93EF930E94C336AF91BF914C
:102EA0000E94CA3684E00E941D2C2896E1E0F0E0E2
:102EB00060E070E0E093490AF0934A0A60934B0A9D
:102EC00070934C0A02C00E94D6350E946A340E9458
:102ED00095341981088126960895E89420F808957C
:102EE0000E94DC320E946A340E94B3340E94823F06
:102EF00011F0E89420F808950E94DC320E946A34B0
:102F00000E94B3340E94823F19F00E946C3602C0C6
:102F10000E94DC32089522970E949A3F06E012E058
:102F200026E032E00E94DC320E946A340E94B33410
:102F30000E94823F11F40C94DC170E946A340E94B4
:102F40009335E091490AF0914A0A0E0F1F1F0E9423
:102F50006A340E949335E091490AF0914A0AEE835F
:102F6000FF830E946A340E949335E091490AF091F0
:102F70004A0A2E0F3F1F40E050E0EE81FF814E17BE
:102F80005F0768F4E42FF52F31970E9439363197A7
:102F9000E00FF11FE081EC934F5F5F4FEECFE1E078
:102FA000F0E060E070E0E093490AF0934A0A609331
:102FB0004B0A70934C0A02C00E94D6350E946A34B4
:102FC0000E9495340E94A13FA0C20E949B3F0E9494
:102FD000DC320E946A340E94B3340E94823F11F4B2
:102FE0000C944F180E946A340E9493350091490A4C
:102FF0000E946A340E9493352091490A30914A0A0E
:103000000E946A340E9493351091490A0E946A34E2
:103010000E9493354091490AE42F0E942133FF9387
:10302000EF930A93EF91FF9109950E94D536A1EA9B
:10303000BDE0AE0FBF1F2D933C930E94D536A7EA8B
:10304000BDE0AE0FBF1F1C930E94D536A9E9BDE0BD
:103050000E9410330E94D536AFE9BDE00E941C33B8
:103060000E94D536A7E9BDE00E941C330E94D536E8
:10307000A9EABDE00E941C330E94D536A8EABDE053
:103080000E941C33E1E0F0E060E070E0E093490A68
:10309000F0934A0A60934B0A70934C0A02C00E9454
:1030A0003F360E946A340E949534EBC20E94DC369F
:1030B0000E946A340E94B3340E94823F11F40C943F
:1030C000BA180E946A340E9493350091490A0E94FE
:1030D0006A340E9493353091490A40914A0A0E940D
:1030E0006A340E9493350E94E0360E949335109115
:1030F000490A0E946A340E9493352091490A0E942D
:10310000E736A7EABDE00E943D33309769F40E949C
:10311000EE364A933A93E0E0EA93EA85FB850E9413
:10312000F2360E9480330DC0E130A0E0FA0749F486
:103130000A934A933A93E885F9850E94F2360E94F1
:1031400086330E94E736A9EABDE00E948C330E94D4
:10315000E736AFE9BDE00E948C33E1E0F0E060E0EB
:1031600070E0E093490AF0934A0A60934B0A709327
:103170004C0A02C00E94F7360E946A340E949534BD
:103180006AC00E94DC360E946A340E94B3340E94F6
:10319000823F11F40C9425190E946A340E949335E1
:1031A0000091490A0E946A340E9493353091490A7D
:1031B00040914A0A0E946A340E9493350E94E03688
:1031C0000E9493351091490A0E946A340E949335F7
:1031D0002091490A0E94E736A7EABDE00E943D33EC
:1031E000309769F40E94EE36EF81F885FA93EA93FE
:1031F000E0E0EA930E94FF360E9491330DC0E13077
:10320000A0E0FA0749F40A93EE81FF81FA93EA936A
:103210000E94FF360E9497330E94E736A9EABDE07C
:103220000E949D330E94E736AFE9BDE00E948C33D7
:10323000E1E0F0E060E070E0E093490AF0934A0AD0
:1032400060934B0A70934C0A02C00E94F7360E94AA
:103250006A340E9495340E94A23F279608950E94E6
:10326000DC320E946A340E94B3340E94823F09F12A
:103270000E946A340E949335E091490AF0E0F0E040
:10328000A3E2B1E00E94B93CA8EABDE00E943D3350
:103290000E9422360E949534E1E0F0E060E070E0A8
:1032A000E093490AF0934A0A60934B0A70934C0AE0
:1032B00002C00E949D350E946A340E949534089590
:1032C00024970E94DC320E946A340E94B3340E9428
:1032D000823FC9F00E94DC320E9446340E94473689
:1032E0000E94813B0E9422360E949534E1E0F0E08A
:1032F00060E070E0E093490AF0934A0A60934B0A59
:1033000070934C0A02C00E949D350E946A340E944C
:1033100095342496089528970E94B3330E94E4328E
:103320000E944B3489F1E12FF0E0A091260AB09180
:10333000270A0E94633CEA0FFB1F0E94753D3197EC
:1033400066277727EA83FB836C837D8300E0011780
:10335000C0F40E94DC320E94463466277727EE8351
:10336000FF83688779870E940437E885F9856A8535
:103370007B85EA5FFD4FFA93EA930E94553B0F5F0E
:10338000E6CF0E94333608C0A6E2BAE0BF93AF93FF
:103390000E94BC35AF91BF91ED93FC930E946A34BB
:1033A0000E949534198108812A96089564970E9495
:1033B000DC320E946A340E94B3340E94823F11F4CE
:1033C0000C942A1A0E946A340E94B334E887F98761
:1033D0006A877B870E946A340E94B334EC83FD8342
:1033E0006E837F830E94DC320E94463466277727F3
:1033F000E88BF98B6A8B7B8B0E94DC320E9446340F
:103400000E940D370E941937D8F4E881F9816A814A
:103410007B810E942437FF93EF93E885F9856A85C5
:103420007B85A889B9898A899B890E94A636EA5F2B
:10343000FD4FE081AF91BF91EC930E942D37E2CF19
:10344000EC81FD816E817F810E942437DF01E0E005
:10345000EC9302C00E943F360E946A340E94953469
:10346000AFC028970E94DC320E946A340E94B334B5
:103470000E94823FA9F00E94DC320E9446340E94E2
:103480003A370E9446340E944736EE81FF816885B4
:103490007985EA5FFD4FFA93EA930E94763B02C07A
:1034A0000E949D350E946A340E9495342EC0289750
:1034B0000E94DC320E94DC320E9446340E943A377D
:1034C0000E94463466277727E883F9836A837B83E3
:1034D000EC81FD816E817F81EA5FFD4FFA93EA9373
:1034E0000E9404370E94643BA0E00E947F3C0E943F
:1034F0006F3CE093490AF0934A0A60934B0A709339
:103500004C0A0E946A340E94953428960895649764
:103510000E94DC320E946A340E94B3340E94823FCF
:1035200011F40C94DA1A0E94DC320E9446346627A9
:103530007727E88BF98B6A8B7B8B0E946A340E9419
:10354000B334E887F9876A877B87E889F9896A89CC
:103550007B89EA5FFD4FFA93EA930E94813B0E94C8
:103560003A370E9446340E940D370E94193708F5F9
:10357000E885F9856A857B85AC85BD858E859F85C7
:103580000E94A636EA5FFD4FFF93EF93E881F98131
:103590006A817B81A889B9898A899B890E941A3CA2
:1035A000EA5FFD4FE081AF91BF91EC930E942D3710
:1035B000DCCF02C00E94D6350E946A340E94953446
:1035C000649608950E949B3F0E94DC320E946A34F8
:1035D0000E94B3340E94823F11F40C943B1B0E9462
:1035E0006A340E9493350091490A10914A0A0E9458
:1035F0006A340E9493354091490A20E030E00E94ED
:10360000D536A3E9BDE0AE0FBF1F0E94663D2E1761
:103610003F0790F40E944137FF93EF93E42F0E94FD
:10362000AD33E757F34FE20FF31FE081AF91BF9146
:10363000EC932F5F3F4FE3CF0E94D536A3E9BDE067
:10364000AE0FBF1F0E94EF330E946A340E94953470
:103650000E94D536A3E9BDE00E941033E1E0F0E01E
:1036600060E070E0E093490AF0934A0A60934B0AE5
:1036700070934C0A02C00E94D6350E946A340E94A0
:1036800095340E94A23F259608950E949A3F0E9479
:10369000DC320E946A340E94B3340E94823F11F4EB
:1036A0000C94E51B0E946A340E9493350091490AEC
:1036B00010914A0A0E946A340E9493355091490A37
:1036C0000E946A340E9493354091490A20E030E01C
:1036D000E52FF0E02E173F0778F4E42F0E94AD337A
:1036E000E757F34FE20FF31FDF010E944137E081FC
:1036F000EC932F5F3F4FECCF0E94D536A5E9BDE09C
:10370000AE0FBF1FE52FF0E0ED93FC930E94D5367E
:10371000A8EABDE0AE0FBF1FE4E0EC930E94D536EF
:10372000A9E9BDE0AE0FBF1FE8EEF3E0ED93FC9317
:103730000E94D536A3E9BDE0AE0FBF1FE1E0F0E087
:10374000ED93FC930E94D536A2E9BDE00E94483774
:10375000F1F00E94D536ACE9BDE00E943D33FF9305
:10376000EF93E081EF93E2E9F0E0FF93EF930E94A3
:10377000D536ADE9BDE00E943D33AF91BF91EA0F70
:10378000FB1FE491AF91EA2BAF91BF91EC930E94A4
:10379000D536AEE9BDE00E943D33FF93EF93E42FB1
:1037A0000E94AD33E757F34FE081AF91BF91EC93A7
:1037B000E1E0F0E060E070E0E093490AF0934A0A4B
:1037C00060934B0A70934C0A02C00E94D6350E9447
:1037D0006A340E9495340E94A13F269608950E9463
:1037E000DC320E946A340E94B3340E94823F99F016
:1037F000E4B7EF700E945F350E949534E1E0F0E09D
:1038000060E070E0E093490AF0934A0A60934B0A43
:1038100070934C0A02C00E94DC320E946A340E94FB
:1038200095340895ECE0F0E80E94753DE050F048D2
:10383000E093260AF093270A689420F820FE05C03A
:103840000E94CD320E947936F9CF0895E4E2EA93DE
:103850000E945628A881B981EC91EA930E945628CB
:10386000E4E30E944D37A181AA930E945628E4E127
:103870000E944D37A281AA930E945628229608954D
:10388000C59AE0914802E17011F0C49A01C0C49851
:10389000E0916500ED7F0E945337E0916500E260A2
:1038A0000E945337EEEFE3B9E6E2F2E00E945B37A5
:1038B000EDEFE3B9EAE2F2E00E945B37EBEFE3B948
:1038C000EEE2F2E00E945B37E7EFE3B9E2E3F2E019
:1038D0000E945B37EFEEE3B9E6E3F2E00E945B376C
:1038E000EFEDE3B9EAE3F2E00E945B37EFEBE3B917
:1038F000EEE3F2E00E945B37EFE7E3B9E2E4F2E0E7
:103900000E945B370895249784E0A0E0B0E0E8E5EA
:10391000F3E00E94A83F0A93ECE5EA930E94562840
:1039200002E00030FCF0E0E0EA930E945628FF2716
:1039300066277727DF01CB01E02FF0E0E7FDFFEFFF
:103940000E94613C0E94753C0E94493CA981BA8159
:103950008B819C810E94293CE983FA836B837C8361
:103960000150DFCFE981FA816B817C81AD81BE811D
:103970000E94703D0881279608950E94F73AE7E07B
:10398000EA93E4E1EA93E9E1EA93E0E0EA930E9452
:103990001028E0E0E8BBE7E3E7BBEFEFE3B9E2B90B
:1039A000E0E0E0936500E2E1E0936400E8E5EDB972
:1039B000E0E0EEB9EFE4F0E060E270E0E0932602D0
:1039C000F09327026093280270932902E0932A0261
:1039D000F0932B0260932C0270932D02E0932E0241
:1039E000F0932F026093300270933102E093320221
:1039F000F09333026093340270933502E093360201
:103A0000F09337026093380270933902E0933A02E0
:103A1000F0933B0260933C0270933D02E0933E02C0
:103A2000F0933F026093400270934102E0934202A0
:103A3000F093430260934402709345020E94401C3D
:103A40000895E0914802E27041F00E94401CE8E4D1
:103A5000F2E0DF01EC91ED7FEC93E62DF0E03097A2
:103A600039F4EEEFE3B9E6E0F2E00E94623753C0CA
:103A7000E130A0E0FA0739F4EDEFE3B9EAE0F2E073
:103A80000E94623748C0E230A0E0FA0739F4EBEF59
:103A9000E3B9EEE0F2E00E9462373DC0E330A0E01F
:103AA000FA0739F4E7EFE3B9E2E1F2E00E946237A6
:103AB00032C0E430A0E0FA0739F4EFEEE3B9E6E112
:103AC000F2E00E94623727C0E530A0E0FA0739F43F
:103AD000EFEDE3B9EAE1F2E00E9462371CC0E630A4
:103AE000A0E0FA0739F4EFEBE3B9EEE1F2E00E946F
:103AF000623711C0E730A0E0FA0761F4EFE7E3B9FD
:103B0000E2E2F2E0FA93EA930E94831CEFEFE3B95A
:103B1000662401C06624A091810CB091820C809132
:103B2000830C9091840CE091850CF091860C60914F
:103B3000870C7091880C0E941F3CDF01CB01E4EFE1
:103B4000F1E060E070E00E94903FC4F4E7E0EA93A7
:103B50000E943128E0934602F0934702E091850CE1
:103B6000F091860C6091870C7091880CE093810C29
:103B7000F093820C6093830C7093840C08950A92E6
:103B80001A926A937A93AA93BA93EA93FA93EFB745
:103B9000EA930A93E6E0E2BFE091850CF091860C8F
:103BA0006091870C7091880CEF5FFF4F6F4F7F4FD4
:103BB000E093850CF093860C6093870C7093880CCF
:103BC000A89500E0013010F00C945F1E0E940933AC
:103BD000A9E9BDE0AE0FBF1F0E94663D309711F40A
:103BE0000C945D1E0E940933A9E9BDE0AE0FBF1F12
:103BF0000E94663D3197ED93FC93309711F00C9441
:103C00005D1E0E940933A8EABDE00E943D33E23008
:103C1000A0E0FA0749F40E940933A8EABDE0AE0F1C
:103C2000BF1FE5E0EC9349C0E330A0E0FA0739F4A8
:103C30000E940933A8EABDE00E941C333EC0E13077
:103C4000A0E0FA0749F40E940933A8EABDE0AE0FEC
:103C5000BF1FE6E0EC9331C0E430A0E0FA0769F55D
:103C60000E940933A8EABDE00E941733A9EABDE02B
:103C70000E941733A2E9BDE00E944837F1F00E948C
:103C80000933ACE9BDE00E943D33FF93EF93E0813F
:103C9000EF93EAE9F0E0FF93EF930E940933ADE977
:103CA000BDE00E943D33AF91BF91EA0FFB1FE4914D
:103CB000AF91EA23AF91BF91EC930F5F83CF09914E
:103CC000E991EFBFF991E991B991A9917991699140
:103CD0001990099018950E946A37E0919C000E9403
:103CE000BA320DD00E94783718950E946A37E9E8F9
:103CF000FCE0FA93EA934DD00E94783718950E9421
:103D00008637E2E0EA17C0F10E948637A230E9F078
:103D1000EA81A0910002EA1739F0A881B981A25E78
:103D2000BE4FAC91A03051F00E948C370E94913769
:103D30000E949837A15EBE4FE2E005C0A881B9811C
:103D4000A15EBE4FE3E0EC9317C00E94A037E930BC
:103D5000A1E0FA0770F40E94A037A881B981EA0FA8
:103D6000FB1FAA81A0830E94A0373196ED93FC939C
:103D700003C00E94A737EC93A881B981A15FBE4F11
:103D8000EC91F0E0A881B981A05FBE4FED93FC9368
:103D9000A5C00E948637A43011F00C94341F0E94F5
:103DA000A037FF93EF93A881B981A45FBE4F0E9413
:103DB000663DAF91BF91AE17BF07B0F4A881B9813E
:103DC0000E94AD37FF93EF930E94A037A881B9817D
:103DD000AE0FBF1FEC91AF91BF91EC930E94A03743
:103DE0003196ED93FC9340C00E94B237B1F00E942F
:103DF000B937FF93EF93E081EF93EAE9F0E0FF93A7
:103E0000EF930E94C037AF91BF91EA0FFB1FE4917F
:103E1000AF91EA23AF91BF91EC93A881B981AA5EDB
:103E2000BE4FAC91E0E0EA1790F4A881B981A85E9A
:103E3000BE4F0E94663DA881B981A05FBE4FED9341
:103E4000FC93A881B981A15EBE4FE1E002C00E944F
:103E5000A737EC93A881B981A65FBE4FE0E0F0E000
:103E6000ED93FC930E94C737229608950E948C37E9
:103E70001196E2E0EC93A881B981A45FBE4FE2E025
:103E8000F0E0ED93FC93A881B9810E94CD37A88121
:103E9000B9810E94D237A881B9810E9491370E94CE
:103EA000B237B1F00E94B937FF93EF93E081EF93FF
:103EB000E2E9F0E0FF93EF930E94C037AF91BF912A
:103EC000EA0FFB1FE491AF91EA2BAF91BF91EC9306
:103ED0000E9498370E94AD37AA81A0832396089547
:103EE0001A930A93EB850E94D937E0910002EC9374
:103EF000AA81BB811296E0E0EC93EA85AA81BB819E
:103F00001396EC93E885AA81BB811496EC93E9851E
:103F1000F070AA81BB811596EC93EF81AA81BB81D9
:103F20001696EC93ED81AA81BB811796EC93EE81F6
:103F3000F070AA81BB811896EC93EC81AA81BB81B9
:103F40001996EC93EAE0F0E00E94DE37AA81BB818B
:103F50001A96EC93AA81BB811B960E94EB37ECE08A
:103F6000F0E00E94F137AA81BB810E94D237AA817A
:103F7000BB810E9491370E94F637B1F00E94FD3755
:103F8000FF93EF93E081EF93E2E9F0E0FF93EF938B
:103F90000E940438AF91BF91EA0FFB1FE491AF91EB
:103FA000EA2BAF91BF91EC930E940B38AA81BB81A1
:103FB0000E94AD37AB85A083198108812C960895A6
:103FC00022970E949D3FEE85AD81BE81EC931196B4
:103FD000E0910002EC93AD81BE811296E1E0EC939A
:103FE000ED85AD81BE811396EC93EB85AD81BE81ED
:103FF0001496EC93EC85F070AD81BE811596EC9330
:10400000EF81AD81BE811696EC93EA85F0E03097A2
:10401000C1F4E6E0F2E0A885B985EA0FFB1FEB8367
:10402000FC8300E0EF810E1758F40E941138FF93D3
:10403000EF930E941938AF91BF91EC930F5FF2CFCD
:1040400066C0E130A0E0FA07D1F4E885F985EB839A
:10405000FC8300E0EF810E1788F40E941138FF9373
:10406000EF93AB81BC811196AB83BC8311970E9407
:104070009A3DAF91BF91EC930F5FECCF48C0E23017
:10408000A0E0FA07D9F4E885F985E050F048EB8321
:10409000FC8300E0EF810E1780F40E941F38AD8191
:1040A000BE81AE0FBF1FEB81FC813196EB83FC8399
:1040B0003197E491EC930F5FEDCF29C0E330A0E09E
:1040C000FA07A1F4E885F985EB83FC8300E0EF8132
:1040D0000E1758F40E941138FF93EF930E9419387D
:1040E000AF91BF91EC930F5FF2CF11C0E430A0E02D
:1040F000FA0769F4E885F985309729F4AD81BE8126
:1041000017964C9204C0E130A0E0FA0701F40E9437
:104110002338FA93EA93EF81F885FA93EA93E0D48F
:104120001E2F2F2F0E942338AD81BE81AE0FBF1FDF
:10413000E22FF0700E9427383896AD81BE81AE0F15
:10414000BF1F1C93EF81F0E03996AD81BE81A45F63
:10415000BE4FED93FC93AD81BE810E94CD37AD8102
:10416000BE810E94D237AD81BE810E949137AD8160
:10417000BE810E942B38D1F0AD81BE810E943038C3
:10418000FF93EF93E081EF93E2E9F0E0FF93EF9389
:10419000AD81BE810E943538AF91BF91EA0FFB1F00
:1041A000E491AF91EA2BAF91BF91EC930E940B3851
:1041B000AD81BE810E94AD37AE85A0830E94A43F31
:1041C0002F96089522970A93E885F0E03097D1F46E
:1041D000E6E0F2E0AE81BF81EA0FFB1FE983FA83DC
:1041E00000E0ED810E1768F40E943A38FF93EF93D8
:1041F0000E941F380E944138AF91BF91EC930F5F2E
:10420000F0CF5DC0E130A0E0FA07B9F4EE81FF81A4
:10421000E983FA8300E0ED810E1770F40E943A38CA
:10422000FF93EF930E941F380E944138AF91BF91D6
:104230000E94B93D0F5FEFCF42C0E230A0E0FA0725
:1042400089F4AE81BF81A050B048FD01EF2FF0E0AE
:10425000FA93EA93ED81FE813796FA93EA930E94EE
:10426000107E2DC0E330A0E0FA07B1F4EE81FF81AB
:10427000E983FA8300E0ED810E1768F40E943A3872
:10428000FF93EF930E941F380E944138AF91BF9176
:10429000EC930F5FF0CF13C0E430A0E0FA0779F49D
:1042A000EE81FF81309739F4AB81BC811796EC9198
:1042B000E093010204C0E130A0E0FA0701F40881B4
:1042C000299608951A930A93E9850E94D937E3E065
:1042D000EC93E885F070AA81BB811296EC93EF8194
:1042E000AA81BB811396EC93AA81BB811496E0E06E
:1042F000EC93EC81AA81BB811596EC93E6E0F0E0AB
:104300000E94DE37AA81BB811696EC93AA81BB81FD
:1043100017960E94EB37E8E0F0E00E94F137AA819F
:10432000BB810E94D237AA81BB810E949137E98567
:10433000AA81BB81A55EBE4FEC93ED81FE81AA816F
:10434000BB81A45EBE4FED93FC930E94F637B1F0A3
:104350000E94FD37FF93EF93E081EF93E2E9F0E0F5
:10436000FF93EF930E940438AF91BF91EA0FFB1FB8
:10437000E491AF91EA2BAF91BF91EC930E940B387F
:10438000AA81BB810E94AD37A985A08319810881CC
:104390002A9608950E949C3FEB85AC81BD81EC93E9
:1043A0001196E6E0EC93EA85F070AC81BD8112963F
:1043B000EC93E985AC81BD811396EC9300E0EE812E
:1043C0000E1730F5E02FEE0F1E2FE12FF0E03496A0
:1043D000AC81BD81EA0FFB1FFF93EF930E9447382A
:1043E0000E944E38AF91BF91EC93E12FF0E03596EB
:1043F000AC81BD81EA0FFB1FFF93EF930E9447380A
:10440000EA5FFD4FE081AF91BF91EC930F5FD7CF93
:104410000E945338FA93EA93EE81FF81FA93EA936C
:104420005FD32E2F3F2F0E945338AC81BD81AE0F3A
:10443000BF1FE32FF070EC930E9459383596AC8182
:10444000BD81AE0FBF1F2C930E9459383696AC81A8
:10445000BD81A45FBE4FED93FC93AC81BD810E94F2
:10446000CD37AC81BD810E94D237AC81BD810E9425
:104470009137EB85AC81BD81A55EBE4FEC93AC81DD
:10448000BD810E942B38D1F0AC81BD810E943038B3
:10449000FF93EF93E081EF93E2E9F0E0FF93EF9376
:1044A000AC81BD810E943538AF91BF91EA0FFB1FEF
:1044B000E491AF91EA2BAF91BF91EC930E940B383E
:1044C000AC81BD810E94AD37AB85A0830E94A33F24
:1044D0002C960895289781E0A0E0B0E0ECE5F3E0A9
:1044E0000E94A83F0E949A3F0E94C737AE85BF85B1
:1044F000A15EBE4FE0E0EC93AE85BF85A25EBE4FED
:104500000E945E3811F00C940D230E94623811F065
:104510000C94DA220E94673811F00C94D9220E9480
:104520007738FF93EF930E947E38AF91BF91EA0FE7
:10453000FB1F0E2F1F2FAE85BF8512960E945E387F
:1045400041F5AE85BF851896EC91FE2FE0E0FF9314
:10455000EF93AE85BF851796EC91F0E0AF91BF91D8
:10456000EA0FFB1F2E2F3F2F0E948438A681AA93AB
:104570003A932A93EA89FB890E948B38ED89FE8958
:10458000A185AA93EE89FF89FA93EA930E94E01F1E
:1045900010C0E130A0E0FA0761F4EE85FF850E94CB
:1045A0008B380E9490380E948438FA93EA930E94D4
:1045B000361F32C0E130A0E0FA0711F50E946738DB
:1045C00031F4AE85BF851296AC91A13009F013C0CD
:1045D0000E947738FF93EF930E947E38AF91BF918E
:1045E000EA0FFB1F0E2F1F2FEE85FF850E948B38D1
:1045F0000E94903802C00E949A380E94A1380CC0D4
:10460000E230A0E0FA0741F40E94A838A23011F08D
:104610000E949A380E94A13815C2E130A0E0FA0742
:1046200011F00C941E250E94623811F00C94BA24EB
:10463000AE85BF85EC91A0910002EA1711F00C94B1
:10464000B9240E94673811F00C94B9240E94AD3847
:10465000FE2FE0E0FF93EF93AE85BF851396EC91BC
:10466000F0E0AF91BF91AE0FBF1FE2E0F0E00E941B
:10467000B93CEF83AE85BF851196EC91F0E0E33055
:10468000A0E0FA07F1F50E94B238FF93EF930E9481
:10469000B938AF91BF910E94BF38AE85BF851296E1
:1046A000EC93E0E0EA87EB870E94C638D8F40E94DA
:1046B000CD380E94D438FF93EF930E94DC380E94DB
:1046C0004E38AF91BF910E94E338FF93EF930E9461
:1046D000DC38EA5FFD4FE081AF91BF91EC930E941F
:1046E000EC38E2CF0E94F2380E94F8380E94033979
:1046F000AE85BF85A45FBE4FED93FC93E1E0EE83F2
:10470000FFC0E430A0E0FA0711F00C94ED230E9402
:10471000B238FF93EF930E94B938AF91BF910E94D6
:10472000BF38AE85BF851296EC93E0E0EA87EB8751
:10473000EC85FD850E941A3910F00C94DE230E944E
:1047400021390E94D438FF93EF930E94DC383396CE
:10475000EA5FFD4FE081AF91BF910E94E338FF9384
:10476000EF930E94DC383296EA5FFD4FE081AF9113
:10477000BF91EC93E885F9853596AE85BF85EA0F44
:10478000FB1FFF93EF930E94DC380E944E38AF91DD
:10479000BF91EC93E885F9853696AE85BF85EA0F23
:1047A000FB1FFF93EF930E94DC38EA5FFD4FE0812F
:1047B000AF91BF91EC930E94EC38BACF0E94F238CF
:1047C0000E94F8380E940339AE85BF85A45FBE4FB2
:1047D000ED93FC93E1E0EE8393C0E630A0E0FA07AE
:1047E000E9F4EF81F0E0EA5FFD4FFF93EF93AE85D0
:1047F000BF851596EC91AF91BF910E9427383196F5
:10480000EA5FFD4FFF93EF93AE85BF851496EC9161
:10481000AF91BF91EC930E94283972C0E031A0E0C3
:10482000FA0711F00C948024AE85BF851696EC91A2
:10483000F0E00E946A3CEC87FD87E0E0EA87EB87C6
:104840000E94C63810F00C9469240E9421390E94FD
:10485000DC38EA5FFD4FFF93EF93E885F9853A96E0
:104860000E943339AF91BF910E9427380E94393995
:10487000FF93EF93E885F98539960E943339AF911C
:10488000BF910E942738A885B985EA0FFB1F329691
:10489000EA5FFD4FFF93EF93E885F98538960E9414
:1048A0003339AF91BF910E942738A885B985EA0FA7
:1048B000FB1F3396EA5FFD4FFF93EF93E885F98581
:1048C00037960E943339AF91BF91EC930E94EC3838
:1048D000B7CFE6E0F0E0FA93EA93E889F989FA9332
:1048E000EA93FED04E2F5F2FE52FF070AE85BF8587
:1048F0001696EC93AE85BF8517964C930E94283987
:10490000EE81E030B1F1AE85BF850E94CD37AE8536
:10491000BF850E94D237AE85BF850E949137AE8594
:10492000BF850E942B38D1F0AE85BF850E943038FC
:10493000FF93EF93E081EF93E2E9F0E0FF93EF93D1
:10494000AE85BF850E943538AF91BF91EA0FFB1F3E
:10495000E491AF91EA2BAF91BF91EC930E940B3899
:10496000AE85BF85AB5EBE4FAC91BB27E091000228
:10497000EC9363C0E130A0E0FA0711F00C94062537
:104980000E94673869F4AE85BF85EC91EF930E9471
:104990004139AF91EA1721F40E94A838A33009F0F9
:1049A00031C0E0E0EA87EB870E94AD38F0E00E947A
:1049B0001A3928F50E94CD380E9447390E943939AA
:1049C000FF93EF93E885F98533960E943339AF91D1
:1049D000BF91EC930E944739A885B985EA0FFB1F68
:1049E000EA5FFD4FFF93EF93E885F98534960E94C7
:1049F0003339AF91BF91EC930E94EC38D5CF0E9430
:104A00004E3902C00E945439EC9317C0E230A0E046
:104A1000FA0799F40E94673849F4AE85BF85EC9196
:104A2000EF930E944139AF91EA1709F003C00E9449
:104A30004E3902C00E945439EC9304C0E230A0E029
:104A4000FA0701F40E94A13F60960895EA81A881C7
:104A5000B981AE5EBE4FEC93F0E0309739F4A88197
:104A6000B981A15FBE4FEAE0EC9338C0E130A0E02D
:104A7000FA0739F4A881B981A15FBE4FE5E0EC9354
:104A80002DC0E230A0E0FA0739F4A881B981A15F16
:104A9000BE4FE3E0EC9322C0E330A0E0FA0719F444
:104AA0000E945A391BC0E430A0E0FA0719F40E94B2
:104AB0005A3914C0E530A0E0FA0719F40E945A39B7
:104AC0000DC0E630A0E0FA0719F40E945A3906C07A
:104AD000E730A0E0FA0711F40E945A3923960895AE
:104AE0000E949C3F0FEF1FEF20E030E0EE81FF813E
:104AF0002E173F0728F5E02FF12FFE2FE0E0FF9360
:104B0000EF93EEE5F3E0FF93EF93E12FF070FF9367
:104B1000EF93E22FF32FAC81BD810E943D33AF9123
:104B2000BF91EA27FB27AF91BF910E946139AF91F6
:104B3000BF91EA27FB270E2F1F2F2F5F3F4FD6CFA6
:104B4000E02FF12F32C00E949C3F0FEF1FEF20E0BB
:104B500030E0EE81FF812E173F0728F5E02FF12F7F
:104B6000FE2FE0E0FF93EF93EEE5F3E0FF93EF938A
:104B7000E12FF070FF93EF93E22FF32FAC81BD8113
:104B80000E945133AF91BF91EA27FB27AF91BF91AC
:104B90000E946139AF91BF91EA27FB270E2F1F2F8B
:104BA0002F5F3F4FD6CFE02FF12F0E94A33F2896D3
:104BB0000895FFFFFFFFFFFFFFFFFFFFFFFFFFFF66
:104BC000FFFFFFFFFFFFFFFFFFFFFFFFFFFFFFFFF5
:104BD000FFFFFFFFFFFFFFFFFFFFFFFFFFFFFFFFE5
:104BE000FFFFFFFFFFFFFFFFFFFFFFFFFFFFFFFFD5
:104BF000FFFFFFFFFFFFFFFFFFFFFFFFFFFFFFFFC5
:105000000E94FC3AEA810E946839EA930E942D3B93
:10501000E881EA930E946D390E940B3B2396089524
:105020000A93EC810E9473390E942D3BE1E00E94BB
:105030006839EE0FEE0FEA930E942D3B0E940B3B66
:105040000A93E2E0EA93ED81EA930E9400280A9332
:10505000E3E0EA93EC81EA930E9400280881259618
:10506000089522970A93EB810E9473390E946D394B
:105070000E94FC3A0F5F0A930E942D3BE1E0EA9305
:105080000E94153BEA83E0E0EA930E94153BE98326
:105090000E940B3BA981BA81E7E00E94403CA5E059
:1050A000B0E00E94E13C088124960895E881EFB9C0
:1050B000779BFECFEFB1219608955F9BFECFACB1F9
:1050C00008955D9BFECFA881ACB921960895A88173
:1050D000B9810E94663D309731F00E947A3931974C
:1050E000AA81A08304C0EA81EA930E9461282396E2
:1050F00008950E948039A885E5E0EA1708F4E8875A
:10510000AEE5B5E0E885F0E00E94633CEA0FFB1FE6
:105110000E94793DA985BA858B859C850E94893E30
:10512000E987FA876B877C8700E0E0E0F0E060E8E1
:105130007FE3EA83FB836C837D83EA81FB816C815F
:105140007D81A985BA858B859C850E944A3F80F028
:10515000AA81BB818C819D81E0E0F0E060E271E496
:105160000E94D73EEA83FB836C837D830F5FE5CF8C
:10517000003029F40E948439E0E3EC932AC0E02F48
:105180000150E03031F1AA81BB818C819D810E9468
:105190008B39EA83FB836C837D83A985BA858B85F4
:1051A0009C850E949B390E9484390E94A139AA8162
:1051B000BB818C819D81FF27662777270E944B3E0C
:1051C0000E94D73EA985BA858B859C850E94A63909
:1051D000D6CFE885E03019F40E94AF392CC00E9488
:1051E0008439EEE2EC93E885E150E887EF5F09F15E
:1051F000A985BA858B859C85E0E0F0E060E271E4EA
:105200000E94D73EE987FA876B877C870E94183E09
:105210001E2F0E9484390E94A139A985BA858B85E9
:105220009C85FF27662777270E944B3E0E94A63960
:10523000DACF0E94AF39198108812D9608952497FD
:105240000E949D3FE0E0F0E060E87FE3EB83FC83B9
:105250006D837E83AA85E5E0EA1708F4EA870A856C
:10526000E02F0150E03019F00E94B439F9CFEB85FE
:10527000FC856D857E850E94823F21F420E00E949E
:10528000B4393AC02A850E94C33909F010F40C944D
:1052900053290E94B4390E94C33920F00E94CE39AC
:1052A0002F5FF9CF15C00E94C33980F4AB85BC8550
:1052B0008D859E85E0E0F0E060E271E40E94D73EDB
:1052C000EB87FC876D877E872150EDCF0E94B43934
:1052D000EB85FC856D857E85A0E0B0E080E09FE3F6
:1052E0000E94893EEB87FC876D877E870E94C339C9
:1052F00018F00E94CE392F5F00E0EA85E017A0F198
:10530000AB81BC818D819E810E948B39EB83FC83B4
:105310006D837E83AB85BC858D859E850E949B3980
:105320000E94DD390E94A139FF27662777270E9456
:105330004B3EAB81BC818D819E810E94D73EAB8567
:10534000BC858D859E850E94843D0E94823EEB87B0
:10535000FC876D877E87E02F0F5FE03071F60E943B
:10536000DD39EEE2EC93C9CF0E94E439A985A08330
:1053700020302CF40E94DD39EDE2EC932195E9E038
:10538000E21764F40E94E439FF93EF93A22FEAE05E
:105390000E94F93CE05DAF91BF91EC930E94E4392B
:1053A000FF93EF93A22FEAE00E94293DE05DAF91C9
:1053B000BF91EC93AF81B885E0E0EC930E94A43FED
:1053C0002F9608951B7FE989EA93EBA1FCA1FA933C
:1053D000EA937DDE403009F04A9508956C970E946B
:1053E0009A3F00E0EEA1FFA13196EEA3FFA3319713
:1053F000E4913E2FE03011F40C94192CE02FF0E0F2
:10540000309739F4353211F401E002C00E94EB39D3
:105410000FC2E130A0E0FA07C9F4353221F40E944E
:10542000EB3900E005C202E0E0E0E98B10E03D323C
:1054300011F411E0FDC13B3219F4EBE2E98BF8C144
:10544000303219F4E0E2E98BF3C104C0E230A0E0AD
:10545000FA0739F440E003E0303311F41068E8C192
:1054600004C0E330A0E0FA0789F4303310F03A3397
:1054700008F006C00E94F239E32FE0534E0FD8C166
:1054800050E03E3211F404E0D3C111C0E430A0E09A
:10549000FA0799F4303310F03A3308F008C010627C
:1054A0000E94F8395E2FE32FE0535E0FC1C13C36F6
:1054B00019F4126005E0BCC106C0E530A0E0FA07AF
:1054C00011F00C94182CE32FF0E0E336A0E0FA077B
:1054D00031F40E94FD39EC910E94043AA8C1E534F0
:1054E000A0E0FA0721F0E536A0E0FA0709F404C0CD
:1054F000E636A0E0FA07F1F5FE017296EE83FF832F
:105500000E94FD390E946A3DE887F9876A877B8798
:10551000DF01CB010E94863F24F0A989AB3229F03C
:105520000EC00E940B3AEDE2E98B17FF04C0E98937
:105530000E94043A04C00E94163AA989A08315FF6C
:1055400055E0363649F40E941D3AEB85FC85FA9306
:10555000EA930E94792809C00E941D3A3A93EC858B
:10556000FD85FA93EA930E941F29FE0172960E941C
:10557000253A22C0E337A0E0FA0739F40E94FD394A
:105580000E94663D0E94253A10C0E037A0E0FA076D
:10559000C1F40E94FD390E94663DEE83FF83FA93B9
:1055A000EA930E948B3B0E2F18601F77503011F04A
:1055B000501708F001C0052F50E0E0E0E88B20E034
:1055C00089C0E436A0E0FA0721F0E936A0E0FA0746
:1055D00011F4146004C0E537A0E0FA07C1F4EAE072
:1055E000E88B11FF0AC0E0E0FAEC6AE97BE3EC87A4
:1055F000FD876E877F870AE02DC0E0E1F7E260E07B
:1056000070E0EC87FD876E877F8705E023C0E83573
:10561000A0E0FA0711F4186006C0E837A0E0FA0726
:1056200011F00C94172CE0E1E88B11FF0AC0E0E0C8
:10563000F0E060E070E1EC87FD876E877F8708E02F
:1056400009C0E0E0F0E160E070E0EC87FD876E8784
:105650007F8704E0503011F01F7701C051E011FF47
:1056600009C00E94FD390E946A3DE887F9876A8770
:105670007B8713C012FF07C00E94FD390E94663D60
:105680000E94753C06C00E94FD390E94663D662757
:105690007727E887F9876A877B8712FF1AC0A88572
:1056A000B9858A859B850E94863F64F4E885F985E3
:1056B0006A857B850E94373CE887F9876A877B8704
:1056C000EDE2E98BE989E03019F00F5F5F5F01C01F
:1056D0001B7F252F10FD14C0041710F4241708F0A9
:1056E0000FC017FF08C012FF04C01B7F398901508B
:1056F00001C030E301C030E20E94EB394150ECCFF1
:10570000051778F4106112FF04C00E94E2290150CD
:105710005150E0E30E94043A403009F041505150AA
:10572000EFCF202FE889E030D1F42030B9F013FF1B
:1057300004C00E94163AE49105C0AE81BF81ED918C
:10574000AE83BF83EA93EBA1FCA1FA93EA930E9494
:105750006728403009F041502150E7CF5FC0EC8509
:10576000FD856E857F85A885B9858A859B850E9484
:10577000FE3C3E2FE9E0E31730F413FF02C0395C32
:1057800001C0395A01C0305D14FD22C0E0E3E317C7
:1057900060F0AC85BD858E859F85A130E0E0BE07B9
:1057A000E0E08E07E0E09E0709F40DC0521710F00C
:1057B00030E309C0421710F010FF01C00EC030E204
:1057C00017FF06C030E3106112FF02C00E94E229F9
:1057D0000E94EB39403009F041502150EC85FD85A5
:1057E0006E857F85A885B9858A859B850E94353D14
:1057F000E887F9876A877B87E889F0E0AC85BD8513
:105800008E859F85662777270E94FE3CEC87FD8763
:105810006E877F870E94823F09F0A1CF10FF07C0EB
:10582000403029F04150E0E20E94043AF9CF00E014
:10583000D9CD0E94A13FA8960895FF92F82E0E940C
:105840002D3A0E94EE29AA81BB81E0E0EC933CC195
:105850000A93AB81BC81EC910E2FE03019F0E0E0AF
:10586000EC9312C0A981BA810E94663D309749F03D
:105870000E94663DE0810E2FE03011F00E947A39DF
:1058800003C00E945D280E2FE02F08812596089501
:1058900027970E949A3FE0E0EB87EC87E989FA8935
:1058A0003196E98BFA8B3197E4912E2FE03011F489
:1058B0000C94592D0E944C3A61F00E94513A2E2FBF
:1058C000E03019F00E944C3A09F401C0F6CF2C8761
:1058D000EFC0253211F00C944E2D40E00E945B3A4F
:1058E000203318F0E9E3E21708F406C00E94F23909
:1058F000E22FE0534E0FF2CF203009F4DAC00E94BD
:10590000513A3E2F0E94613AD1F7303009F4CAC0B3
:105910003C87403009F44FEF50E0E22FF0E0E336EF
:10592000A0E0FA0741F40E94663A0E94513AA02F83
:10593000B12FEC93AFC0E337A0E0FA07E9F40E947F
:10594000663AE42F4150E03091F00E94513A2E2FF8
:10595000E03019F00E944C3A09F009C01F930F93F0
:105960000F5F1F4FE22FAF91BF91EC93EACFA02FB3
:10597000B12FE0E0EC938EC0EC36A0E0FA0719F40A
:1059800051E00E945B3AE1E0EA87E22FF0E0E43682
:10599000A0E0FA0721F0E936A0E0FA0719F4E0E008
:1059A000EA8704C0E537A0E0FA0711F43AE00DC039
:1059B000E837A0E0FA0711F430E107C0E532A0E0D3
:1059C000FA0709F46BC0EB8575C0E0E0EE83EF8366
:1059D000E887E987E42F4150E030B9F10E94513A5D
:1059E0002E2FAE2FE0E2EA17B8F4EA85E03039F462
:1059F0002D3219F4EFEFEA87EDCFE1E0EA872033AB
:105A000058F0213610F0275505C0213410F02753E7
:105A100001C02053231710F02C8717C0E32FF0E0AC
:105A2000AE81BF8188859985662777270E94C13C12
:105A3000DF01CB01E22FF0E0662777270E941A3CB6
:105A4000EE83FF8368877987C5CFEA85F0E0E7FDBD
:105A5000FFEFAE81BF81888599850E94753C0E94C9
:105A6000C13CEE83FF8368877987503059F00E94EC
:105A7000663AEE81FF8168857985A02FB12F0E945B
:105A8000703D08C00E94663AEE81FF81A02FB12FC1
:105A9000ED93FC93EB85EF5FEB870AC00E94513AD0
:105AA000E21731F0EB85E03011F4EFEF03C001C0F5
:105AB000F5CEEB850E94A13F63960895FF92F82EE4
:105AC0000E942D3A0E94482C198108812496FF904B
:105AD0000895E991F991699179913097604070400A
:105AE00042F4E095F0956095709500243196601D24
:105AF000701D089566277727A991B9918991999189
:105B0000E1E0FF27AE1BBF0B860B970B18F0329618
:105B1000671FF8CF6695F795E7950895E991F99194
:105B2000699179917F7708952497EC81FD816E8149
:105B30007F810E94823F29F4E0E0F0E060E070E0C5
:105B4000E7C1EC81FD816E817F81A885B9858A8559
:105B50009B850E94093FE883F9836A837B830E94C7
:105B6000823F29F4E0E0F0E060E070E0D1C1A8817C
:105B7000B9818A819B810E948A3F4CF4E881F98136
:105B80006A817B810E947F3D0E94073C08C0E881BA
:105B9000F9816A817B810E947F3D0E940D3CE883F0
:105BA000F9836A837B83AC81BD818E819F810E9452
:105BB000D73EA885B9858A859B850E94843D0E9431
:105BC000823EA6C10E948039AE81BF8188859985B9
:105BD0000E948A3F2CF0EFEFFFEF6FE77FEF8AC064
:105BE000EE81FF81688579850E947F3DEDB7FEB724
:105BF0003197FA93EA931F930F930E94CE3D0F9132
:105C00001F91EE83FF8368877987AE81BF81888586
:105C10009985E3EFF4E065E37FE30E944A3F60F497
:105C2000EE81FF81688579850E94893EEE83FF833E
:105C30006887798701501040AE81BF81888599853A
:105C40000E946F3A7F936F93FF93EF93EE81FF81F2
:105C500068857985A0E0B0E080E89FE30E94893EF6
:105C6000AF91BF918F919F910E94093F0E94783A16
:105C7000A6E2B2E485E69FE30E94D73EDF01CB01B6
:105C8000EEE4F1E164E570E40E94843D0E94823E0E
:105C9000AE81BF81888599850E94D73E7F936F939F
:105CA000FF93EF93AA81BB818C819D81EDE4F1E1AB
:105CB00064ED7FE30E94843D0E94823EAF91BF91DC
:105CC0008F919F910E94093F7F936F93FF93EF9372
:105CD000E02FF12FA8E1B2E781E39FE30E94753C3A
:105CE0000E944B3E0E94D73EAF91BF918F919F91F2
:105CF0000E94893E198108812A96089528971A934F
:105D00000A93AA85BB858C859D85E0E5FCEA6EEA51
:105D100072EC0E944A3F28F4E0E0F0E060E070E0BE
:105D200095C0EA85FB856C857D850E94823F29F4BC
:105D3000E0E0F0E060E87FE389C0AA85BB858C8560
:105D40009D85E8E1F2E761EB72E40E944A3F09F0C9
:105D500010F40C94B02EEFEFFFEF6FE77FE776C003
:105D6000AA85BB858C859D85EBE3FAEA68EB7FE32A
:105D70000E94D73EEA87FB876C877D870E947F3D24
:105D80000E94073C0E94183E0E2F1F2FE02FF12F7C
:105D9000AA85BB858C859D850E94753C0E944B3EE3
:105DA0000E940C360E94843D0E94823E0E94783AF6
:105DB000ADE6BCE48CE69DE30E94D73EA6EAB3EED6
:105DC00086EE90E40E94893EAE81BF8188859985E8
:105DD0000E94D73EEE83FF8368877987EA81FB8143
:105DE0006C817D81A8E2BDE886EA91E40E94893E4B
:105DF000EA83FB836C837D83EE81FF8168857985EF
:105E0000AA81BB818C819D810E94893EA3EFB4E071
:105E100085EB9FE30E94D73E7F936F93FF93EF93B1
:105E2000AE81BF8188859985EA81FB816C817D8106
:105E30000E94823EAF91BF918F919F910E94093F36
:105E40000E947F3D1A930A930E94E13D19810881C7
:105E50002E9608952497E885F9856A857B850E94AA
:105E6000823F29F4E0E0F0E060E070E051C0A885F6
:105E7000B9858A859B850E948A3F9CF4EC81FD81CF
:105E80006E817F810E94823F29F4E0E0F0E060E8CB
:105E90007FE33EC0E885F9856A857B850E94873A65
:105EA00037C0EC81FD816E817F81DE010E94183E4A
:105EB0000E94703DE881F9816A817B810E944B3E9E
:105EC000DF01CB01EC81FD816E817F810E94903FDB
:105ED00029F0E0E0F0E060E070E01AC0E885F985C4
:105EE0006A857B850E94EF3D0E94873AE887F987A3
:105EF0006A877B87E881E17029F4E885F9856A85FE
:105F00007B8506C0E885F9856A857B850E94EF3D23
:105F10002C96089524970A9300E0AD81BE818F816D
:105F20009885E3E8F9EF62E27EE30E94D73EED83D5
:105F3000FE836F8378870E947F3D0E94073CAD817E
:105F4000BE818F8198850E94953AAD81BE818F81F7
:105F50009885E0E0F0E060E07FE30E944A3F09F0CE
:105F600010F40C94B62F0E94953A01E0AD81BE81E9
:105F70008F819885E0E0F0E060E87EE30E944A3F90
:105F800009F010F40C94CE2FE0E0F0E060E07FE345
:105F90000E94823EED83FE836F837887003011F08C
:105FA0000E949E3A0E94A93AE983FA836B837C831C
:105FB000A1EBB4EC86E292E40E94D73EDF01CB0174
:105FC000EDE1F5EE6DE272E40E94843D0E94823EB6
:105FD000A981BA818B819C810E94D73EACE4B3E554
:105FE00084E091E40E94893EAD81BE818F819885D5
:105FF0000E94D73E7F936F93FF93EF93E981FA81DD
:106000006B817C81A1E1BDEE8EED9FE30E94893E14
:10601000A981BA818B819C810E94D73EAEE5BBE706
:1060200088EA9FE30E94893EAF91BF918F919F9133
:106030000E94093F34C1A881B9818A819B81EBED1F
:10604000FFE069EC7FE30E94823E0E947F3D0E9458
:106050008A2F6AC12497EC81FD816E817F810E9425
:106060007F3D0E941B30E883F9836A837B830E9413
:10607000823F89F4AC81BD818E819F810E948A3FDD
:106080002CF4EFEFFFEF6FE77FE74BC0EFEFFFEF91
:106090006FE77FEF46C0EC81FD816E817F810E94BA
:1060A0007F3D0E948A2FDF01CB01E881F9816A815F
:1060B0007B810E94093F35C02497EC81FD816E8170
:1060C0007F81AC81BD818E819F810E94D73EE88314
:1060D000F9836A837B83A5E6B0ED8BEC90E40E94A4
:1060E000B43AAC81BD818E819F810E94D73E7F935F
:1060F0006F93FF93EF93E881F9816A817B81A0E040
:10610000BDE689E291E40E94893EA881B9818A8135
:106110009B810E94B43AAF91BF918F919F910E9451
:10612000093F28960895A881B9818A819B81EDEC69
:10613000F3E164ED7EE30E944A3F48F4E881F9818F
:106140006A817B810E947F3D0E945C30EDC0A88106
:10615000B9818A819B81EAE7F2E86AE170E40E94F2
:106160004A3F09F010F40C94C230E881F9816A8149
:106170007B81A0E0B0E080E89FE30E94BD3A0E94EE
:10618000C33AD2C0A881B9818A819B810E946F3AAB
:106190007F936F93FF93EF93E881F9816A817B810D
:1061A000A0E0B0E080E89FE30E94893EAF91BF91FC
:1061B0008F919F910E94BD3AABEDBFE089E49FE3D0
:1061C0000E94893EB1C024970A9300E0AD81BE8150
:1061D0008F819885E0E0F0E060E87FEB0E944A3F25
:1061E00058F0E0E0F0E060E87FE30E944A3F19F0F9
:1061F00010F00C94FC3005C0EFEFFFEF6FE77FE786
:106200004EC0AD81BE818F8198850E94863F1CF46F
:106210000E949E3A01E00E94A93AA0E0B0E080E826
:106220009FE30E94843D0E94823E0E947F3D0E9427
:10623000A23BE983FA836B837C83AD81BE818F812E
:106240009885E3EFF4E065E37FE30E944A3F09F0BD
:1062500010F40C943831ED81FE816F817885A9812D
:10626000BA818B819C810E94CC3A0E94C33A0AC0B9
:10627000E981FA816B817C81AD81BE818F819885B6
:106280000E94CC3AE983FA836B837C83003019F057
:106290000E94EF3D04C0E981FA816B817C81088115
:1062A00029960895A881B9818A819B81E0E0F0E078
:1062B00060E87FEB0E944A3F58F0E0E0F0E060E8E1
:1062C0007FE30E944A3F19F010F00C94683105C03A
:1062D000EFEFFFEF6FE77FE727C0E881F9816A8181
:1062E0007B810E947F3D0E94E3300E94C33A1CC024
:1062F000A881B9818A819B810E94863F4CF0E88108
:10630000F9816A817B810E947F3D0E9493300CC09D
:10631000E881F9816A817B810E94EF3D0E947F3D87
:106320000E9493300E94EF3D249608952A970E9480
:106330009A3FE0E0E887E987EA87EB87A889B9898F
:10634000EC914E2F0E94613A19F00E94D23AF6CF9A
:10635000E0E0EF834B3219F40E94D23A06C04D328E
:1063600021F4E1E0EF830E94D23AE0E05E2F4E2F6D
:1063700008891989A889B989EC910E94D83A49F409
:10638000A889B989AC91EEE20E947F3C4E2FE030A3
:1063900021F0542B0E94D23AEDCF28893989503010
:1063A00019F10E94DD3AA889B989AC91AE32E1F0C9
:1063B0000E94E33AA885B9858A859B85FF276627D1
:1063C00077270E944B3E0E94893EDF01CB01E0E02F
:1063D000F0E060E271E40E94093FE887F9876A878C
:1063E0007B870E94DD3ADFCFE0E0F0E060E87FE30A
:1063F000EC87FD876E877F87A889B9891197A88B5D
:10640000B98BA017B107D0F00E94E33AAC85BD85E7
:106410008E859F85FF27662777270E944B3E0E9427
:10642000D73EA885B9858A859B850E94893EE887E5
:10643000F9876A877B870E94E83ADECFA22FB32FC5
:106440002F5F3F4F4C91453619F0453409F067C036
:10645000E0E05E2FEE83A22FB32FAC91AD3221F49A
:10646000E1E0EE832F5F3F4FA22FB32F2F5F3F4F0F
:10647000EC914E2F0E94D83A31F00E94F839E40F87
:10648000E0535E2FF1CFE6E2E51768F4EF81E030EC
:1064900029F0EFEFFFEF6FE77FEF4AC0EFEFFFEF7D
:1064A0006FE77FE745C040E2E0E0F0E060E87FE3CF
:1064B000EC87FD876E877F874030A9F0EC85FD85EE
:1064C0006E857F85AC85BD858E859F850E94D73E74
:1064D000EC87FD876E877F87E52FE42311F00E940C
:1064E000E83A4695E9CFEE81E03059F0EC85FD853C
:1064F0006E857F85A885B9858A859B850E94093F21
:106500000AC0EC85FD856E857F85A885B9858A855D
:106510009B850E94D73EE887F9876A877B87EF8152
:10652000E03011F00E940B3AE885F9856A857B8599
:106530000E94A13F62960895E091AC0DF091AD0DDF
:106540006091AE0D7091AF0DADE6BEE486EC91E4C6
:106550000E94C13CEE59F8486F4F7F4FE093AC0D5D
:10656000F093AD0D6093AE0D7093AF0DE62FF72F46
:10657000FF770895EA93E9E8FCE0FA93EA93089537
:10658000E881F0E0309708950E94753DE050F048B2
:10659000E093260AF093270A0895A6E2BAE00E9443
:1065A000663D3296ED93FC930895E091260AF091B2
:1065B000270AE491F0E00895A6E2BAE00E94663D61
:1065C0003496ED93FC930895A6E2BAE00E94663DEE
:1065D0003196ED93FC930895E42FF52F0E94683CCB
:1065E000EA5FFD4F0895E42FF52FE770F070EA0F92
:1065F000FB1FE4910895A6E0B2E0EE0FFF1FAE0F7F
:10660000BF1F0895A6E0B2E00E94633CAE0FBF1F1B
:106610000895A02FBB27E3E2F1E00E94B93C089562
:10662000AE0FBF1FE0E0F0E0ED93FC930895AE0FD6
:10663000BF1FE0E0EC93EDCFAE0FBF1FE0E0EC93A7
:106640000895F0E0A2E0B2E0EE0FFF1FAE0FBF1F13
:106650000E94663D0895E091260AF091270A32963D
:106660000E94753D0895A12FBB27E3E2F1E00E944F
:10667000B93C0895E491EC93F6CFAE0FBF1FEC91B7
:10668000F0E00895A02FB12FE3E2F1E00E94B93CC1
:106690000895AE0FBF1F0E94663DDF01E22FF32F6A
:1066A0000895EA0FFB1FE491F0E00895AE0FBF1FBD
:1066B0000E94663DE20FF31FE491EA930895E0E043
:1066C000EA93E0CFF695E7953196EE0FFF1FEA0FBC
:1066D000FB1F0E94753DFA93EA930895F695E7959E
:1066E0003296EE0FFF1FEA0FFB1F0E94753DFA93D3
:1066F000EA93C8CF3696EA0FFB1FE491EA93C2CF24
:10670000E757F34FFA93EA930C94701FE757F34F50
:10671000FA93EA930C946221AE0FBF1FE1E0EC9371
:106720000895E757F34FFA93EA930C94E01FE75765
:10673000F34FFA93EA930C94CA21AE0FBF1FE2E025
:10674000EC930895AE0FBF1FEC91EF5F0895E757EC
:10675000F34FFA93EA930C946A22F0E0A3E2B1E0DB
:106760000E94B93C08951A930A9326CF34970E9449
:10677000753D0E2F1F2F0895E02FF12F0E94683CCA
:10678000E050F84FEA5FFD4F0895A2E9B0E0E02F36
:10679000F12FE770F070EA0FFB1FE4910895E02FEE
:1067A000F12F0E94683CEA5FFD4F089534970E94E4
:1067B000753D3197EA5FFD4FE0810895F0E066276F
:1067C0007727E093490AF0934A0A60934B0A709343
:1067D0004C0A089534970E94753D31970CCF0E9462
:1067E000663D66277727E093490AF0934A0A60934B
:1067F0004B0A70934C0A089534970E94753D319767
:1068000001CFAAE9B0E0E02FF12FE770F070EA0FB6
:10681000FB1FE491089534970E94753D3197EA5F1C
:10682000FD4FDF01E091490AF0914A0A60914B0A5D
:1068300070914C0AEC93089534970E94753D3197FE
:10684000A6E0B2E0EE0FFF1FAE0FBF1FE091490AB6
:10685000F0914A0A60914B0A70914C0AED93FC93B7
:10686000089534970E94753D3197A6E0B2E00E94EA
:10687000633CAE0FBF1FE091490AF0914A0A609154
:106880004B0A70914C0A0E94703D089534970E9403
:10689000753D319708953197E491E1501E2FE091B5
:1068A000260AF091270A3396E491F0E0A3E5BAE0D6
:1068B000EE0FFF1FAE0FBF1FED91FD910995E09107
:1068C000490AF0914A0A60914B0A70914C0A0E9461
:1068D000823F0895E091260AF091270A3396E491C9
:1068E000F0E00895A3E5BAE0EE0FFF1FAE0FBF1F63
:1068F000ED91FD910995E091490AF0914A0A609164
:106900004B0A70914C0AAA81BB818C819D810895AC
:10691000EA81FB816C817D81E093490AF0934A0A08
:1069200060934B0A70934C0AD5CFA7E6BAE0EE0FFE
:10693000FF1FAE0FBF1FED91FD91099508950E94B5
:10694000663DDF01E12FF0E00E94633CEA0FFB1F90
:106950000895ED93FC93E091260AF091270A0E9496
:10696000753DF0780895A3E5BAE0EE0FFF1FAE0F76
:10697000BF1FED91FD910995E091490AF0914A0AF6
:1069800060914B0A70914C0A0895A6E2BAE00E9409
:10699000663D3497ED93FC939DCFA881B9818A81A0
:1069A0009B810E94893CFF2766277727E093490A4D
:1069B000F0934A0A60934B0A70934C0A8BCFA881DC
:1069C000B9818A819B810E94913CFF2766277727A6
:1069D000E093490AF0934A0A60934B0A70934C0A79
:1069E00079CF0E94A93CFF2766277727E093490AC1
:1069F000F0934A0A60934B0A70934C0A6BCF0E9443
:106A0000B13CFF2766277727E093490AF0934A0AAB
:106A100060934B0A70934C0A5DCF0E94993CFF270C
:106A200066277727E093490AF0934A0A60934B0A56
:106A300070934C0A4FCFA881B9818A819B810E94B3
:106A4000A13CFF2766277727E093490AF0934A0A7B
:106A500060934B0A70934C0A3DCFA3E5BAE0EE0F6A
:106A6000FF1FAE0FBF1FED91FD910995A091490A3F
:106A7000B0914A0A80914B0A90914C0AE0E0F0E014
:106A800060E070E008950E94893CFF276627772721
:106A9000E093490AF0934A0A60934B0A70934C0AB8
:106AA00019CF0E94913CFF2766277727E093490A78
:106AB000F0934A0A60934B0A70934C0A0BCFFF275E
:106AC00066277727E093490AF0934A0A60934B0AB6
:106AD00070934C0AFFCE0E94F707E0914D0AF091A7
:106AE0004E0A60914F0A7091500AE883F9836A83D5
:106AF0007B830E94F707E0914D0AF0914E0A609166
:106B00004F0A7091500A08950E94F707A0914D0A0C
:106B1000B0914E0A80914F0A9091500AE0E0F0E067
:106B200060E070E00895A3E5BAE0EE0FFF1FAE0F3E
:106B3000BF1FED91FD9109950895A6E2BAE00E946C
:106B4000663D3896ED93FC930895E0934D0AF093DB
:106B50004E0A60934F0A7093500A0E947308E1E056
:106B6000F0E060E070E0E093490AF0934A0A609335
:106B70004B0A70934C0A08950E94663DDF01E12F95
:106B8000F0E031960E94633CEA0FFB1F08950E94DB
:106B9000F707E0914D0AF0914E0A60914F0A70910B
:106BA000500AAA81BB818C819D810895A6E2BAE03A
:106BB0000E94663D3C96ED93FC9308950E94F70772
:106BC000E0914D0AF0914E0A60914F0A7091500A7F
:106BD000E883F9836A837B830C94F707E881F98162
:106BE0006A817B810E947F3DE0914D0AF0914E0ABF
:106BF00060914F0A7091500A0E947F3D08950E9453
:106C0000F707E0914D0AF0914E0A60914F0A70919A
:106C1000500A0E947F3D08950E94843D0E94823E5A
:106C2000DF01CB01E0E0F0E060E07FE308950E9447
:106C3000183EE093490AF0934A0A60934B0A709316
:106C40004C0A48CE66277727E093490AF0934A0A10
:106C500060934B0A70934C0A3DCEA6E2BAE00E94C4
:106C6000663D38960895A6E2BAE00E94663D3496E5
:106C70000895E20FF31FDF01E42FF52F0895A6E238
:106C8000BAE00E94663D7096ED93FC9308956627E6
:106C90007727E883F9836A837B83EA5FFD4FFA9362
:106CA000EA930895E091490AF0914A0A60914B0AEB
:106CB00070914C0AEA5FFD4FFA93EA930895E02F32
:106CC000F0E0A5E0B0E00E94B93C0895F0E0EE0FDE
:106CD000FF1FE85DF54F0895E091260AF091270A1D
:106CE0000E94753DE050F048E093260AF093270A91
:106CF000089532970E94753DABE7BAE0EE0FFF1F93
:106D0000AE0FBF1FED91FD9109950895E091490ADD
:106D1000F0914A0A0E94633CEC83FD83AC81BD8103
:106D20001497E881F9816A817B810E94A63D0895CC
:106D3000E091490AF0914A0A0E94633CE883F98392
:106D4000A881B98114970E94913D08950E941A3C30
:106D5000A881B9818A819B810E941A3C0895E981AA
:106D6000FA816B817C81EA5FFD4FFA93EA93089583
:106D7000EA0FFB1FFA93EA93E9E4FAE06627772724
:106D80000E947F3D0895E12FF0E0A5E0B0E00E9471
:106D9000B93C0895EA0FFB1FFA93EA93EE81FF8155
:106DA000688579850E947F3D0895A42FBB27E3E283
:106DB000F1E00E94B93C089522970E949B3FFCCBD2
:106DC000E091490AF0914A0AED83FE8383CDA22F18
:106DD000BB27E3E2F1E00E94B93C08950A93E0E0AA
:106DE000EA930895FA93EA931A93E22FB6CCA6E2B7
:106DF000BAE00E94663D7496ED93FC9308954A9321
:106E00003A931A93E22FA9CCEA81FB816C817D81B0
:106E1000EA5FFD4FFA93EA93089566277727EC8798
:106E2000FD876E877F87E0E0E883E983EA83EB8371
:106E30000895EC81FD816E817F81A881B9818A816D
:106E40009B810E94953F0895AC85BD858E859F8569
:106E50000E941A3CEA5FFD4F0895E881F9816A813A
:106E60007B81EF5FFF4F6F4F7F4FE883F9836A832A
:106E70007B83089566277727EC83FD836E837F836A
:106E80009BCBE22FF32FE00FF11FEA5FFD4F089538
:106E9000AE0FBF1FEC91E1700895EA930E9456284F
:106EA000E881F9810895E0936500EAE0F0E0FA9363
:106EB000EA930C94963BFA93EA930E94261CEFEF18
:106EC000E3B90895FA93EA930E94831CEFEFE3B9C4
:106ED000639408950A921A92FA926A937A938A9323
:106EE0009A93AA93BA93EA93FA93EFB7EA93089521
:106EF000E991EFBFF991E991B991A991999189919E
:106F000079916991F990199009900895A881B981B2
:106F1000A15EBE4FAC910895EA81A881B981EC933E
:106F20000895A65FBE4FE1E0F0E0ED93FC93089575
:106F3000E0916200E860E0936200A881B981089561
:106F4000A881B981A65FBE4F0E94663D0895A881C1
:106F5000B981A15EBE4FE0E00895AB5EBE4FEC91FB
:106F6000F0E00895A881B981A75FBE4FEC91E17070
:106F70000895A881B981AD5EBE4FEC91F0E008950F
:106F8000A881B981AC5EBE4FEC91F0E00895E0912C
:106F90006200E77FE09362000895A15EBE4FE4E0E7
:106FA000EC930895A05FBE4FE8EEF3E0ED93FC9301
:106FB0000895AA81BB81EC9311960895FA93EA9300
:106FC000EC81FD81FA93EA930E9470250E2F1F2F0A
:106FD000E12FF07008950C93AA81BB81A45FBE4F8E
:106FE0000895ED93FC93AA81BB81D7CFAA81BB8181
:106FF000A75FBE4FEC91E1700895AA81BB81AD5EA1
:10700000BE4FEC91F0E00895AA81BB81AC5EBE4F0B
:10701000EC91F0E00895E0916200E860E093620096
:107020000895E02FF0E03796AD81BE81EA0FFB1F97
:107030000895AB81BC81ED91AB83BC830895E02FB3
:10704000F0E037960895EF81F0E037960895EC93DD
:10705000EF81F0E00895A75FBE4FEC91E1700895D5
:10706000AD5EBE4FEC91F0E00895AC5EBE4FEC918A
:10707000F0E00895E981FA813196E983FA83319746
:107080000895AB81BC81AE0FBF1FEC910895E12F35
:10709000F0E0AF81B885EA0FFB1F08953196EA5FF3
:1070A000FD4FE0810895EE81F0E0EE0FFF1F349672
:1070B0000895EE81F0E0EE0FFF1F0895EC91F0E0EF
:1070C00030970895AE85BF85A05EBE4FF7CFAE85E1
:1070D000BF85A65FBE4F0E94663DFA93EA93E8899A
:1070E000F989FA93EA930E94702530970895AE8546
:1070F000BF851596EC91FE2FE0E00895AE85BF8523
:107100001496EC91F0E00895EE85FF85A181AA9395
:10711000EF85F8890895A381AA931A930A93089595
:10712000E989FA89A681AA93EA89FB89FA93EA9305
:107130000C94E220AE85BF85A15EBE4FE6E0EC93E5
:107140000895AE85BF85A05EBE4FE0E0EC93089544
:10715000AE85BF851196AC910895AE85BF85129618
:10716000EC910895AE85BF851496EC91FE2FE0E07A
:107170000895AE85BF851596EC91F0E00895EA0F6D
:10718000FB1FEC87FD87EE0FFF1F0895EC85FD8543
:10719000AA85BB85AE17BF070895EA85FB85EE0F6C
:1071A000FF1FE887F9870895E885F9853396AE854E
:1071B000BF85EA0FFB1F0895EF81F0E0A885B98530
:1071C000EA0FFB1F0895EC93E885F9853496AE85A8
:1071D000BF85EA0FFB1F0895EA85FB853196EA8794
:1071E000FB870895EC85FD85EE0FFF1F339608950C
:1071F000FA93EA93E889F989FA93EA930E94702551
:107200004E2F5F2FEFCFAE85BF85AE0FBF1FE52F8F
:10721000F070EC93EC85FD85EE0FFF1F3496AE8584
:10722000BF85AE0FBF1F4C93EC85FD85EE0FFF1F92
:1072300035960895F695E795AA85BB85AE17BF07E5
:107240000895EA85FB850E94633CE887F9870895E5
:10725000AE85BF85A45FBE4FE8E0F0E0ED93FC9300
:10726000E1E0EE830895AE85BF85AE0FBF1FEC91C0
:107270000895A885B985EA0FFB1F3196EA5FFD4F97
:107280000895AE85BF85A55EBE4FEC910895AE858D
:10729000BF85A45EBE4F0E94663D0895AE85BF8542
:1072A000A05EBE4FE0E00895AE85BF85A15EBE4FF3
:1072B000E6E00895A881B981A15FBE4FE2E0EC93BA
:1072C0000895EE0FFF1FEA0FFB1F0E94753D089502
:1072D000EA930E942D3BE98108950E942D3BE0E056
:1072E000EA930C942D3BEE0FE0690E2F0E94FC3ABE
:1072F0000A9308950E94663D3196ED93FC9308959C
:1073000024971A930A930895AE81BF811196AE8394
:10731000BF8311970895E0E0F0E060E271E40E941D
:10732000093FA0E0B0E080E09FE30E94893E0E9418
:107330007F3D0C94073C0E94093F0E94183E1E2F7F
:107340000895E12FE05DEC93E12F08950E94843DC4
:107350000E94823EE987FA876B877C870895AE8119
:10736000BF81E0E0EC930895AB81BC818D819E816B
:10737000E0E0F0E060E271E40E94D73EEB83FC8342
:107380006D837E830895EB81FC816D817E81AB8569
:10739000BC858D859E850E944A3F0895AB85BC853E
:1073A0008D859E85E0E0F0E060E271E40E94093F97
:1073B000EB87FC876D877E870895AF81B88511962E
:1073C000AF83B88711970895EF81F8853196EF83E1
:1073D000F887319708953A93EBA1FCA1FA93EA93C9
:1073E0000C946728A42FEAE0EA9FE02D4E2F089521
:1073F000A52FEAE0EA9FE02D0895ACA1BDA1149766
:10740000ACA3BDA314960895EA93EBA1FCA1FA9353
:10741000EA930C946728E885F9856A857B850E9444
:10742000EF3DE887F9876A877B870895EE81FF81C2
:107430003196EE83FF8331970895E885F9856A8553
:107440007B850E947F3D5A930895EE83FF83FA93D4
:10745000EA930E94813B0E2F089522971A930A9374
:10746000DE010E94163C0A2F1B2FDE0116960E9499
:10747000163C0E94663DEA83FB83DE0114960E945F
:10748000163C0E94663DFA93EA931A930A93FE0112
:107490003696FA93EA9308952A930E944B3BE03084
:1074A0000895FE013C96FA93EA93EF85F889FA93E2
:1074B000EA930C94282CE989FA892591E98BFA8BB7
:1074C0000895EA930E944B3BE0300895AF85B88958
:1074D0001497AF87B88B14960D911C910895E0E036
:1074E000F0E060E87FE30E94843D0E94823E0895C0
:1074F000EE83FF8368877987AE81BF818885998510
:107500000E94D73EEA83FB836C837D8308950E94AB
:107510007F3D0E94E22DAC81BD818E819F810E94C2
:10752000D73E0E947F3D0C947E2E0E94843D0E9497
:10753000823EED83FE836F8378870895ED81FE811F
:107540006F8178850E94EF3DED83FE836F8378879E
:107550000895ED81FE816F817885AD81BE818F8137
:1075600098850E94D73E08950E94D73EAEE4BFE8BA
:107570008AE491E40E94893E08950E94093F0E9496
:107580007F3D0C945C30ABEDBFE089EC9FE30E9443
:10759000843D0E94823E08950E94093F0E947F3DE3
:1075A0000C949330E889F9893196E88BF98B08952A
:1075B000EA930E94433BE0300895E889F9893197C6
:1075C000E88BF98B0895A889B989EC91E053089567
:1075D000AC85BD858E859F85E0E0F0E060E271E4DA
:1075E0000E94D73EEC87FD876E877F870895C798F6
:1075F000C698BF9ABE9815C0BE98BF98EE270000E7
:10760000B69B0895B79B089504D0BE9A02D0BF9A46
:10761000E1E06BE107C0BE9ABF9A03D0BF98F9DFE3
:10762000BE9865E36A95F1F7089578E0BF98F9DFB1
:107630008894B6990894BF9AF4DFEE1F7A95B1F753
:107640007991772311F4BE9801C0BE9AE2DFBF980A
:10765000E8DFBF9ADEDFBE98DCCFE99178E0EE0F7D
:1076600010F4BE9801C0BE9ADCDFBF98DADFBF9A83
:107670007A95A9F7BE98CDDFBF98D3DFE1E0B69940
:10768000EE27BF9A0895E1E0F991F03310F0FA3354
:1076900008F0EE270895E1E0F991F03229F0F93091
:1076A00010F0FE3008F0EE270895E991F991A991C4
:1076B000B991CD016D916623E9F7119761916D93B1
:1076C0006623E1F7FC010895E991F991A991B99137
:1076D0006D917191671721F46623D1F7EE27089514
:1076E000671BE1F3E1E008F4E2500895E991F991B4
:1076F000A991B991CD0161916D936623E1F7FC01E8
:107700000895A991B991EE27FF276D91662311F095
:107710003196FBCF0895AA27BB27E991F9910590EF
:10772000002011F01196FBCFFD010895E991F99128
:10773000309639F080EA9FE00197F1F7A8953197EC
:10774000C9F7089524975F939F81992311F4289690
:1077500022C312F4289625C34F9342E48E81BD8143
:10776000AC8188839983AA83BB83FD01BC01AC8172
:10777000BD818E819F814DD388819981AA81BB81F2
:10778000C8D24DD27A9531D288819981AA81BB81A4
:10779000AE27A87F21F4BF178607970729F04A95DF
:1077A00019F0DF01CB01DDCF4F915F91289608954D
:1077B0007B816A81F981E88177FB770F67FD7160D2
:1077C000972F9E5781F078F0983190F4AA27BB2725
:1077D000882708948795B795A7959A95D1F7EA23B6
:1077E000FB23682305C0E8947727EE27FF27662749
:1077F0006F77769508F4606877F9A991B9918991C6
:107800009991EA17FB076807790797FB0895D0DF7E
:1078100009F40895F6F79FEB05C0CADF09F408954F
:10782000F6F39FE3AA27BB2780E873C20024AF0DBD
:10783000B01D0895EA0FFB1F681F791F0895EA1B0A
:10784000FB0B680B790B0895EA23FB23682379234C
:107850000895EA2BFB2B682B792B0895EA27FB2749
:10786000682779270895E095F09531960895E09579
:10787000F09560957095EF5FFF4F6F4F7F4F0895C4
:10788000EE230E2EFD0121F0F595E7950A94E1F720
:107890000895EE230E2EFD01BC0131F0EE0FFF1F07
:1078A000661F771F0A94D1F70895EE230E2EFD016F
:1078B000BC0131F075956795F795E7950A94D1F776
:1078C0000895EE0FFF1FEE0FFF1FEE0FFF1F08952D
:1078D000F695E795F695E795F695E7950895FE2FC9
:1078E000FF0FFF0B6F2F7F2F08956F2F660F660B13
:1078F000762F0895E095F095609570950895EA17B4
:10790000E1E009F0EE270895EA17E1E009F4EE2737
:107910000895EA17FB0768077907E1E009F0EE2709
:107920000895EA17FB0768077907E1E009F4EE27F5
:107930000895EA17FB0768077907E1E00CF4EE27E2
:107940000895AE17BF0786079707E1E00CF4EE270E
:107950000895AE17BF0786079707E1E00CF0EE2702
:107960000895EA17FB0768077907E1E00CF0EE27B6
:107970000895FA9FF02DEB9FF00DEA9FE02DF10D99
:1079800008957A9F702D6B9F700DF89F700DE99F81
:10799000700D6A9F602D710DFB9F600D711DE89F3A
:1079A000600D711D8827FA9FF02D610D781FEB9FE8
:1079B000F00D611D781FEA9FE02DF10D681F781F03
:1079C000089563D0D6DF0EF44EDF08956CD0D9DF72
:1079D0000EF44DDF0895002498E0AA0F001C0E1A43
:1079E00010F40E0E01C0A1609A95B9F7EA2FA02DF0
:1079F00008953FD0F0DF0EF4E19508953F934F9343
:107A00005F93002411243327442750E2AA0FBB1FA1
:107A1000881F991F001C111C331F441F0E1A1F0AB8
:107A2000360B470B28F40E0E1F1E361F471F01C0D2
:107A3000A1605A9559F7FD01BC01D001832F942F05
:107A40005F914F913F9108952ED0D8DF0EF40FDF54
:107A50000895E894A7FF02C0A1956894E7FDE19519
:107A6000BADFEA2F0EF4E1950895C8DFFD01BC01ED
:107A70000895E894E7FF02C0E1956894A7FF04C069
:107A8000A19500F8039400FA0895E894F7FF02C066
:107A9000EADE6894B7FF06C0A095B095119600F88D
:107AA000039400FA0895E89477FF02C0E0DE68943A
:107AB00097FF0BC00024A095B095809590951196E6
:107AC000801D901D00F8039400FA0895ED91FC913B
:107AD00011970895ED91FD916D917C911397089503
:107AE000ED93FD936D937C9308950590F491E02DB3
:107AF00008950590159065917491F00108957A9319
:107B00006A93FA93EA930895182E862F612D192E01
:107B1000972F712D1B2EBF2FF12D1A2EAE2FE12D79
:107B20000895129603D07F2F6E2F1297119602D0D0
:107B3000FE2F1197E199FECFFF93FFB7F894AEBBEC
:107B4000BFBBE09AEDB3FFBFFF9108950AD0129634
:107B50000E2E1F2EE62FF72F04D0E02DF12D1297B9
:107B6000089507D01196EF93EF2F03D0EF9111975F
:107B70000895E199FECF9FB7F894AEBBBFBBE09AE2
:107B80008DB3E81719F0EDBBE29AE19A9FBF089513
:107B9000992761916D930197E1F70895A991B991A2
:107BA000E991F9916991799177FB660F771F8827A1
:107BB0007E57880B7D938C937EE7769567957EF054
:107BC0000895A991B991E991F9916991799177FB1A
:107BD000660F771F7A0F769567950EF008953097A8
:107BE0006040704009F07058089550E8572711F42C
:107BF0005F93D1C05F3F31F0660F000C57956795DA
:107C0000752F08955F9300200AF0CBC0BEC050E8E6
:107C1000192E1522880F991F9527550F879550E823
:107C2000072E0522660F771F7527550F6795089554
:107C30005F93F5DF703818F07F3F08F4ACC056E171
:107C4000571B92F45195583028F0EFEFFFEF6FEF8C
:107C50007FE71AC077275523B9F0EE0FFF1F661F85
:107C6000771F5A95D1F710C07727583028F0EF2F9B
:107C7000F62F672F5850F9CF552331F07695679539
:107C8000F795E7955A95D1F700200AF4F0DD5F915A
:107C90000895689401C0E894309760407040B1F056
:107CA000002426F0772312F40094E1DD172E7EE104
:107CB000112032F07A95EE0FFF1F661F111CF9CFCD
:107CC000EF2FF62F612D5F9390DF5F9108955E2F68
:107CD000EA2FA52F5F2FFB2FB52F562F682F852F4B
:107CE000572F792F952F502D012C152E0895EA0F1F
:107CF000FB1F681F0895E095F0956095EF5FFF4FBB
:107D00006F4F08955F9383DF903871F150E8152627
:107D100004C05F937CDF903839F1703821F1572F20
:107D2000591B13F112F4D3DFFACF583118F0AA27F8
:107D3000BB278827583028F0AB2FB82F88275850FA
:107D4000F9CF552329F08695B795A7955A95D9F778
:107D5000502D512562F0CBDF38F46795F795E79504
:107D6000739513F41EC0B3DF40DF5F910895EA1BE3
:107D7000FB0B680B81F010F40094BDDF6623A2F3C7
:107D8000EE0FFF1F661F7A95CBF7EFEFFFEF6FE760
:107D90007FEF5F910895EE27FF27662777275F9192
:107DA0000895EFEFFFEF6FE77FE75F9108955F932F
:107DB0002EDF703881F3903871F301240894791F15
:107DC00023F44CF300200AF3ECCF3F934F9311249C
:107DD00033274427552798E1330F441F551FEE1FC3
:107DE000FF1F661F30F43A0F4B1F581FE11DF11D96
:107DF000611D9A9589F74F913F9166232AF0550F9F
:107E0000EE1FFF1F661F02C07395E3F2EEDE5F9167
:107E100008955F93FCDE703819F4112012F6B5CF87
:107E2000903809F4B8CF01240894970B1BF4D4F3CD
:107E30000020F4CF792F6695F795E7958695B7954D
:107E4000A7954F9311244427552798E1AE17BF07F4
:107E5000860728F0AE1BBF0B860B089401C08894E0
:107E6000111C441F551FAA1FBB1F881F9A9571F72D
:107E7000E12DF42F652FA695E91FF91F691F4F917A
:107E800066232AF0EE0FFF1F661F7A955BF2ADDEC8
:107E90005F91089599239AF0772342F0971748F05D
:107EA00029F4AE17BF07860720F031F09894889424
:107EB00008959894089408951894889408957723C1
:107EC000C2F7971798F3A9F7EA17FB07680788F333
:107ED00099F3ECCFDFDFE1E011F008F0EE27089531
:107EE000D9DFE1E011F008F4EE270895D3DFE1E0F7
:107EF00009F008F0EE270895CDDFE1E009F008F47D
:107F0000EE270895309760407040089510978040A4
:107F10009040089500240A160B06080609060895E5
:107F2000EA17FB07680779070895AE17BF078607AA
:107F3000970708955A934A933A932A931A930A9368
:107F400008955D814C813B812A81198108810895C2
:107F5000AC0FBD1F05900D928A95E1F70895FFFFC4
:107F6000FFFFFFFFFFFFFFFFFFFFFFFFFFFFFFFF21
:107F7000FFFFFFFFFFFFFFFFFFFFFFFFFFFFFFFF11
:107F8000FFFFFFFFFFFFFFFFFFFFFFFFFFFFFFFF01
:107F9000FFFFFFFFFFFFFFFFFFFFFFFFFFFFFFFFF1
:107FA000FFFFFFFFFFFFFFFFFFFFFFFFFFFFFFFFE1
:107FB000FFFFFFFFFFFFFFFFFFFFFFFFFFFFFFFFD1
:107FC000FFFFFFFFFFFFFFFFFFFFFFFFFFFFFFFFC1
:107FD000FFFFFFFFFFFFFFFFFFFFFFFFFFFFFFFFB1
:107FE000FFFFFFFFFFFFFFFFFFFFFFFFFFFFFFFFA1
:107FF000FFFFFFFFFFFFFFFFFFFFFFFFFFFFFFFF91
:108000009DACE20329002C002D00DA032A00E103D5
:108010000000000000000000504143353235305F61
:10802000300000000000000000005900002B000399
:1080300041493101000000080000000000034149EF
:108040003202000000080000000000034149330331
:108050000000000800000000000341493404000053
:108060000008000000000003414935050000000839
:10807000000000000003414936060000000800002F
:10808000000000034149370700000008000000001D
:108090000003414938080000000800000000000EFD
:1080A0004149315F46696C746572486967682100AF
:1080B0000000044F000000000D4149315F46696C2B
:1080C0007465724C6F77220000000400000000000D
:1080D0000C4149315F4D6F64654761696E23000053
:1080E000000420000000000C4149315F52657365B7
:1080F00072766564240000000400000000000E4158
:1081000049325F46696C746572486967682500008A
:1081100000044F000000000D4149325F46696C7455
:1081200065724C6F77260000000400000000000C10
:108130004149325F4D6F64654761696E27000000F9
:108140000420000000000C4149325F5265736572E3
:10815000766564280000000400000000000E41491C
:10816000335F46696C74657248696768290000006E
:10817000044F000000000D4149335F46696C74658F
:10818000724C6F772A0000000400000000000C41D0
:1081900049335F4D6F64654761696E2B00000004D1
:1081A00020000000000C4149335F52657365727610
:1081B00065642C0000000400000000000E414934FA
:1081C0005F46696C746572486967682D0000000439
:1081D0004F000000000D4149345F46696C746572C0
:1081E0004C6F772E0000000400000000000C414995
:1081F000345F4D6F64654761696E2F000000042095
:10820000000000000C4149345F5265736572766569
:1082100064300000000400000000000E4149355F9A
:1082200046696C7465724869676831000000044FE4
:10823000000000000D4149355F46696C7465724C61
:108240006F77320000000400000000000C41493547
:108250005F4D6F64654761696E3300000004200064
:108260000000000C4149355F5265736572766564A4
:10827000340000000400000000000E4149365F4653
:10828000696C7465724869676835000000044F00C6
:108290000000000D4149365F46696C7465724C6F91
:1082A00077360000000400000000000C4149365FF2
:1082B0004D6F64654761696E37000000042000005F
:1082C00000000C4149365F5265736572766564380B
:1082D0000000000400000000000E4149375F4669BD
:1082E0006C7465724869676839000000044F0000CB
:1082F00000000D4149375F46696C7465724C6F77B9
:108300003A0000000400000000000C4149375F4DB6
:108310006F64654761696E3B000000042000000047
:10832000000C4149375F52657365727665643C00A5
:1083300000000400000000000E4149385F46696CEF
:10834000746572486967683D000000044F000000D2
:10835000000D4149385F46696C7465724C6F773E19
:108360000000000400000000000C4149385F4D6F20
:1083700064654761696E3F00000004200000000052
:108380000C4149385F526573657276656440000040
:1083900000040000000000094C6F63616C54656DBF
:1083A00070210000000500000000000A4149735FD1
:1083B000427566666572110200000200000000004E
:1083C0000F4149735F4368616E67655365747570EB
:1083D0001202000002010000000001000064000120
:1083E000000000001A010000010000000901000067
:1083F000010001020003003A000000040000000038
:10840000FFFFFFFFFFFFFFFFFFFFFFFFFFFFFFFF7C
:10841000FFFFFFFFFFFFFFFFFFFFFFFFFFFFFFFF6C
:10842000FFFFFFFFFFFFFFFFFFFFFFFFFFFFFFFF5C
:10843000FFFFFFFFFFFFFFFFFFFFFFFFFFFFFFFF4C
:10F000000C944F790C9400780C9400780C94007850
:10F010000C9400780C9400780C9400780C94007890
:10F020000C9400780C9400780C9400780C94007880
:10F030000C9400780C9400780C9400780C94007870
:10F040000C94F9790C9400780C9400780C94007866
:10F050000C9400780C9400780C9400780C94007850
:10F060000C9400780C9400780C9400780C94007840
:10F070000C9400780C9400780C94567A0C940078D8
:10F080000C949A7A0C9400780C940078010204088D
:10F0900010204080FEFDFBF7EFDFBF7F0000C0C106
:10F0A000C1810140C30103C00280C241C60106C044
:10F0B0000780C7410500C5C1C4810440CC010CC014
:10F0C0000D80CD410F00CFC1CE810E400A00CAC1D4
:10F0D000CB810B40C90109C00880C841D80118C0C4
:10F0E0001980D9411B00DBC1DA811A401E00DEC144
:10F0F000DF811F40DD011DC01C80DC411400D4C134
:10F10000D5811540D70117C01680D641D20112C053
:10F110001380D3411100D1C1D0811040F00130C023
:10F120003180F1413300F3C1F28132403600F6C143
:10F13000F7813740F50135C03480F4413C00FCC113
:10F14000FD813D40FF013FC03E80FE41FA013AC0D3
:10F150003B80FB413900F9C1F88138402800E8C103
:10F16000E9812940EB012BC02A80EA41EE012EC043
:10F170002F80EF412D00EDC1EC812C40E40124C033
:10F180002580E5412700E7C1E68126402200E2C153
:10F19000E3812340E10121C02080E041A00160C063
:10F1A0006180A1416300A3C1A28162406600A6C143
:10F1B000A7816740A50165C06480A4416C00ACC113
:10F1C000AD816D40AF016FC06E80AE41AA016AC0D3
:10F1D0006B80AB416900A9C1A88168407800B8C1C3
:10F1E000B9817940BB017BC07A80BA41BE017EC043
:10F1F0007F80BF417D00BDC1BC817C40B40174C033
:10F200007580B5417700B7C1B68176407200B2C152
:10F21000B3817340B10171C07080B041500090C1A2
:10F2200091815140930153C052809241960156C042
:10F2300057809741550095C1948154409C015CC012
:10F240005D809D415F009FC19E815E405A009AC1D2
:10F250009B815B40990159C058809841880148C002
:10F26000498089414B008BC18A814A404E008EC142
:10F270008F814F408D014DC04C808C41440084C132
:10F2800085814540870147C046808641820142C052
:10F2900043808341410081C1808140400000F89457
:10F2A000EE27ECBBF1E0F5BFF2E0F5BFE0936C00B8
:10F2B000F8E1F1BDE1BD8DE0A2E0BB27ED938A95B9
:10F2C000E9F780E090E1A0E0B1E0ED930197E9F784
:10F2D000ECE9F2EF85919591009761F0A591B591D8
:10F2E00005901590BF01F00105900D920197E1F78F
:10F2F000FB01F0CFEFEFEDBFE0E1EEBFC0E0D2E009
:10F300000C94BF7B09801A80EB81FC81B881B0939B
:10F310006800E895E0916800E170E1F725960895AE
:10F320001A930A93F8940E944D7CE3E00E94587C63
:10F3300000E010E00038E0E01E07A8F4E02FF12F15
:10F34000EE0FFF1FFA93EA93AC81BD81ED91FD9121
:10F35000AC83BD83FA93EA93E1E0EA930E94827959
:10F360000F5F1F4FE7CF0E944D7CE5E00E94587C65
:10F37000789419810881269608950E94B27C0FEF37
:10F380001FEF20E030E0EE81FF812E173F0758F598
:10F39000E02FF12FFE2FE0E0FF93EF93ECE9F0EF89
:10F3A000FF93EF93E12FF070FF93EF93E22FF32F92
:10F3B000AC81BD81AE0FBF1FEC91F0E0AF91BF916A
:10F3C000EA27FB27AF91BF91EE0FFF1FEA0FFB1F4C
:10F3D0000E94A97CAF91BF91EA27FB270E2F1F2F18
:10F3E0002F5F3F4FD0CFE02FF12F0E94B77C2896A0
:10F3F00008956A937A93AA93BA93EA93FA93EFB72C
:10F40000EA93E6E0E2BFE0911703F0911803609100
:10F41000190370911A03EF5FFF4F6F4F7F4FE09317
:10F420001703F09318036093190370931A03A895B8
:10F43000E0910E03F0910F03309779F1AEE0B3E065
:10F440000E94A57C3197ED93FC93309731F5E091C4
:10F450001303F0E0E230A0E0FA0721F4E5E0E093E6
:10F4600013031BC0E330A0E0FA0721F4E0E0E093CF
:10F47000130313C0E130A0E0FA0721F4E6E0E093C3
:10F4800013030BC0E430A0E0FA0739F4E0E0E093A6
:10F490001303E09314030E94657CE991EFBFF99197
:10F4A000E991B991A9917991699118950E946B7C24
:10F4B0000A9300919C00A0911303E2E0EA1778F10F
:10F4C000A0911303A230A1F0031571F40093000280
:10F4D000E1E0F0E0E0930903F0930A030E94727CFC
:10F4E000E2E0E093130303C0E3E0E093130317C0EB
:10F4F000E0910903F0910A03E930A1E0FA0760F412
:10F50000E0910903F0910A03E050FE4F0083A9E067
:10F51000B3E00E94787C03C0E0E0E0931303E09145
:10F520000D03F0E0E0930E03F0930F0309910E94A6
:10F530007E7C18950E946B7CA0911303A43069F522
:10F54000A9E0B3E00E94A57CFF93EF93ABE0B3E0AA
:10F550000E94A57CAF91BF91AE17BF0770F4E091F8
:10F560000903F0910A03E050FE4FE081E0939C0014
:10F57000A9E0B3E00E94787C10C00E94657CE0E0C6
:10F58000E0931303E0E0F0E0E0930903F0930A0353
:10F59000E0916200E77FE09362000E947E7C189514
:10F5A000E881E0930002E2E0E0930102E2E0F0E0B3
:10F5B000E0930B03F0930C03E4E0E0931303E8EE15
:10F5C000F3E0E0930E03F0930F03E1E0F0E0E0934B
:10F5D0000903F0930A030E94857CE881E0939C0074
:10F5E0002196089522970E94B37CEC85E093000257
:10F5F00030920102E1E0E0930202EB85E093030226
:10F60000E985E0930402EA85E0930502ED81E09349
:10F610000602E885F0E0E230A0E0FA07A9F4EE8106
:10F62000FF81EB83FC8300E0ED810E1768F4E02F8F
:10F630000E948B7CEB81FC813196EB83FC833197BC
:10F64000E491EC930F5FF0CFED81F0E037960E94EC
:10F65000917C1E2F2F2FED810E948B7CE22FF0706A
:10F66000EC93ED81F0E03896E050FE4F1083ED8191
:10F67000F0E03996E0930B03F0930C03E4E0E093A1
:10F680001303E8EEF3E0E0930E03F0930F03E1E0E1
:10F69000F0E0E0930903F0930A030E94857CEC8577
:10F6A000E0939C000E94B87C2D960895AA81A23018
:10F6B00079F4E981F070FA93EA93E7E0F2E0FA93E3
:10F6C000EA930E949079E981F070EBBBE0E0E5BB42
:10F6D000239608950E94B27CE0E0E0931303E0914A
:10F6E0001403F0E0309711F00C94BB7BE091090318
:10F6F000F0910A030E94917C309711F00C94BB7B2F
:10F70000B0910502A0E0E0910402F0E0EA0FFB1FD7
:10F710000E2F1F2FE0910202F0E03097E1F4B0913C
:10F720000802E0910702F0E0EA0FFB1F2E2F3F2FA7
:10F73000E0910102EA93E0910602EA933A932A9358
:10F74000E0910302EA931A930A93E0910902EA9383
:10F750000E94F27A10C0E130A0E0FA0761F4E09173
:10F760000302EA931A930A930E94567BE0910102E6
:10F77000EA930E94D07A0E94B77C24960895249739
:10F78000E0E0EBBBEFEFEABBE0E0E5BBEFEFE4BBB3
:10F79000E0EFE2BBE3E0E1BBE0B3E095AE2FEA2FA0
:10F7A000E295EF703E2E332011F40C94D97B0C942B
:10F7B0000000E0E0E8BBE7BBE3B9E2B9BAD0B9D0FA
:10F7C000E1E0E0936500E0E1E0936400E4E0E3BFA2
:10F7D000E6E0E2BFE0E0E1BFE1E0E7BFE0E0E093C8
:10F7E0007D00E0E8E8B9E0E0E0BDE2E0E0939B0006
:10F7F000E8EDE0939A00E6E0E0939D00E0E0E0931E
:10F800009800EFE0E0939900929AE2E0E0930D0314
:10F810007894EFEFEBBBE5BBE0911703F091180391
:10F820006091190370911A03E883F9836A837B83DB
:10F83000E881F9816A817B81A0911703B091180357
:10F840008091190390911A030E94A07CEAEFF0E0E6
:10F8500060E070E00E94AD7C94F4E894919B689421
:10F86000A2B3A1F9A2BBE0911703F0911803609134
:10F87000190370911A03E883F9836A837B83E0910B
:10F880001303F0E0309731F0E530A0E0FA0711F40F
:10F890000E946A7BCDCF2496FFCFEC81FD81FE2FA5
:10F8A000E0E0FA93EA93E0E0F0E0FA93EA93089557
:10F8B000EA930E948279E0E0F0E0FA93EA93FA9307
:10F8C000EA93E1E1EA930C948279E0916500EF70AC
:10F8D000E09365000895AA93BA93EA93FA93EFB779
:10F8E000EA930895E0916200E860E0936200089571
:10F8F0000E94A57C3196ED93FC930895E991EFBFAA
:10F90000F991E991B991A9910895E0916500E061BB
:10F91000E0936500E7CFF0E03796E050FE4FDF015F
:10F920000895FA93EA93E0E0F2E0FA93EA930C94F4
:10F93000BD79EFE0E0936200E8E0E09361000895B4
:10F94000AE1BBF0B860B970B0895ED91FC911197A1
:10F9500008950590F491E02D0895EA17FB076807D4
:10F96000790708953A932A931A930A9308953B814D
:10F970002A81198108810895FFFFFFFFFFFFFFFF24
:10F98000FFFFFFFFFFFFFFFFFFFFFFFFFFFFFFFF87
:10F99000FFFFFFFFFFFFFFFFFFFFFFFFFFFFFFFF77
:10F9A000FFFFFFFFFFFFFFFFFFFFFFFFFFFFFFFF67
:10F9B000FFFFFFFFFFFFFFFFFFFFFFFFFFFFFFFF57
:10FC00000C94000009801A80EB81FC81B881B093CC
:10FC10006800E895E0916800E170E1F725960895A5
:10FC20001A930A93F894EC81FD81FE2FE0E0FA9399
:10FC3000EA93E0E0F0E0FA93EA93E3E0EA930E94CB
:10FC4000027EE0E0F0E0FA93EA93FA93EA93E1E1CE
:10FC5000EA930E94027E00E010E00038E0E01E0718
:10FC6000A8F4E02FF12FEE0FFF1FFA93EA93AC8177
:10FC7000BD81ED91FD91AC83BD83FA93EA93E1E000
:10FC8000EA930E94027E0F5F1F4FE7CFEC81FD8158
:10FC9000FE2FE0E0FA93EA93E0E0F0E0FA93EA93D3
:10FCA000E5E0EA930E94027EE0E0F0E0FA93EA9356
:10FCB000FA93EA93E1E1EA930E94027E7894198133
:10FCC000088126960895FFFFFFFFFFFFFFFFFFFF5C
:10FCD000FFFFFFFFFFFFFFFFFFFFFFFFFFFFFFFF34
:10FCE000FFFFFFFFFFFFFFFFFFFFFFFFFFFFFFFF24
:10FCF000FFFFFFFFFFFFFFFFFFFFFFFFFFFFFFFF14
:10FD0000FFFFFFFFFFFFFFFFFFFFFFFFFFFFFFFF03
:00000001FF
